:020000040800F2
:20000000880C00202D0200083502000837020008390200083B0200083D02000800000000A6
:200020000000000000000000000000003F020008410200080000000043020008251C000896
:20004000470200084702000847020008470200084702000847020008470200084702000818
:200060004702000847020008470200084702000847020008470200084702000847020008F8
:200080004702000847020008470200084702000847020008470200084702000847020008D8
:2000A00047020008470200084702000847020008470200080000000000000000470200085A
:2000C000470200084702000847020008470200084702000847020008470200084702000898
:2000E00047020008470200080000000000000000000000000000000000000000000000005E
:2001000000000000470200080000000047020008000000000000000047020008470200089B
:2001200047020008470200084702000847020008470200080000000000000000000000002A
:20014000470200084702000847020008000000004702000847020008470200084702000868
:200160004702000847020008470200080000000047020008470200080000000000000000EA
:2001800047020008470200084702000800F002F800F03CF80AA090E8000C82448344AAF108
:2001A0000107DA4501D100F031F8AFF2090EBAE80F0013F0010F18BFFB1A43F0010318472F
:2001C0005C2000007C200000103A24BF78C878C1FAD8520724BF30C830C144BF04680C608F
:2001E000704700000023002400250026103A28BF78C1FBD8520728BF30C148BF0B6070471F
:200200001FB501F0CCFF1FBD10B510BD00F058F81146FFF7F5FF01F0B9FF00F076F803B4A1
:20022000FFF7F2FF03BC00F07BF800000948804709480047FEE7FEE7FEE7FEE7FEE7FEE7A7
:20024000FEE7FEE7FEE7FEE704480549054A064B70470000FD1C00088D01000888060020B4
:20026000880C002088080020880800204FF0000200B5134694469646203922BFA0E80C5047
:20028000A0E80C50B1F12001BFF4F7AF090728BFA0E80C5048BF0CC05DF804EB890028BFFC
:2002A00040F8042B08BF704748BF20F8022B11F0804F18BF00F8012B704770477047704766
:2002C000754600F029F8AE4605006946534620F00700854618B020B5FFF7B6FFBDE82040E2
:2002E0004FF000064FF000074FF000084FF0000B21F00701AC46ACE8C009ACE8C009ACE889
:20030000C009ACE8C0098D4670470446AFF300802046FFF784FF0000004870472806002095
:2003200001491820ABBEFEE726000200704700F0D5F9FCE710B500F089F9012812D00A4CD5
:20034000207801280ED101F0E1FCD4E90112114401F5FA61884205D300202070BDE8104072
:2003600000F0D6B910BD000038000020044910B50120087000F006F8BDE81040FFF7DABFBC
:200380003800002010B5044C2078012802D101F0BDFCA06010BD00003800002010B500F0D8
:2003A000A1F901F0BBFC01F0D5FA00F0F1FB0549086000F08DF900F039F9BDE81040FFF726
:2003C000D5BF00004400002010B500F087F901F0FDFC00F043F9BDE81040FFF7ABBF000085
:2003E0002DE9FF410446984615460E46684601F04FF902984FF47A71B0FBF1F21648002312
:200400004FF4806700EB430C10F813109CF801C06144491C6143B2FBF1FC01FB1C2CBCF1BF
:20042000000F12D1B2FBF1F189B23180491EB9420BD210F8131000EB43002970417888F8E5
:200440000010012004B0BDE8F0815B1CDBB2122BD8D30020F6E70000F021000870B58EB03C
:2004600000242A48ADF828408DF82C408DF8304000680CAB0BAA00880AA940F010054FF45C
:200480007A70FFF7ADFF18B9B62121A0FFF74FFF2748264901260160047644768476C67653
:2004A000047744778460C4609DF82C10491E090401619DF830100905A1F580114161BDF8F6
:2004C0002810416000F0DBFC002D02DB6905194804E0042000EBC501164840420A0C89B2B9
:2004E0000594CDE90021CDE90646010C80B2CDE9021004940E20CDE9086069460C4800F0AC
:20050000CDFB0B4800F058FD0EB070BD440000202E2E5C447269766572735C4F70656E4265
:200520004C545C63616E2E630000000000640040640000200400E0FF70B50E46104988B0E7
:200540000025096803466A4609880E4841F01004294600F01AFC80B9002C05DB0098A042AC
:200560000BD1029830B108E00198A04205D10298042802D104980125307008B0284670BD9D
:200580004400002064000020154A10B5126888B013880022002B02DB0093029202E001933B
:2005A00004230293CDE90321024606AB69460D4800F016FB002811D101F0A8FB00F13204E2
:2005C00006E000BF00F08AF801F0A0FBA04205D80448069900F0E0FC0028F3D108B010BD91
:2005E00044000020640000207047000006480078042807D2DFE800F00606020408207047E9
:200600003F207047812070474800002006480078042807D2DFE800F0060602040820704791
:200620003F207047812070474800002010B501F08DFCFFF713FF044C0220207001F03EFA72
:200640000020207010BD00004800002010B5002401F08AFC00B10124204610BD38B56946B0
:200660000D48FFF769FF0D4C012806D1022020709DF80010084801F081FC6946064801F06B
:2006800055FA012806D1002020709DF80010024801F074FC38BD00008C0000204800002002
:2006A00070B50A4D06460C462878022803D1E1B23046FFF769FF287818B9E1B2304601F0B0
:2006C0008BFABDE8704001F029BD000048000020AFF300804FF4FA7001F0EAB8AFF300807D
:2006E00001F00EB9AFF3008072B6704762B6704770B515460E46044606E000BF16F8010B95
:2007000004F8010BFFF7EAFF6D1EADB2F6D270BD10B501F021F9002818D000F01DF8002806
:2007200014D0FFF761FF00F073FC01F033FB01F00FF9074908400749086001F009F9446819
:20074000FFF7D4FFA446BDE81040604710BD000080FFFF1F08ED00E010B54FF090414FF4F3
:2007600000700969884301D0002010BD01F09AF8012010BD144A117F1448012901D003292C
:200780000FD1036823F400730360036843F400630360036823F400630360036843F400735C
:2007A0000360022901D003290BD1016841F480510160016821F480510160016841F48061D3
:2007C00001600020107770471400002000200240C107054803D0416941F0040141614169B0
:2007E00041F48031416170470020024008494A69C0B222F47E7242EAC0004861486940F066
:2008000002004861486940F4803048617047000000200240054910B54C6944F001044C6128
:200820000260BFF36F8F436010BD000000200240094A10B55469402344F480245461EFF329
:20084000108272B610C910C05B1E13F0FF03F9D182F3108810BD00000020024070B5054641
:2008600000F0CAFC0646134C08E0681C06D000F0C3FC801BA84201D3032070BD2069C00331
:20088000F3D420690C4908400CD00C494A6802434A60810F01D0A169A161810000D020615A
:2008A000012070BD2069C00701D001202061002070BD000000200240FAC302001400002085
:2008C0002DE9F04104464D0A00686D021F4690460E46401C05D12946204600F0BDF80028F6
:2008E00026D02068A84205D02946204600F0C4F804001FD02068301A051946464FF4007810
:2009000015F10405FFF7EAFE281B001F404508D32168204601F5007100F0AEF8040009D05F
:20092000251D16F8010B05F8010B7F1EEAD10120BDE8F0810020FBE70A4810B50068401CE6
:2009400004D0084800F0DEF8002809D006480068401C04D0044800F0D5F8002800D00120A4
:2009600010BD000014030020100100202DE9F0432E4A0127131A4A1E85B0934209D3C60A0E
:200980002B4AF602964204D34218521EB2F1016F03D3002005B0BDE8F083801B0844C0F301
:2009A000CF25400501D06D1CADB200F011FC21494FF40040086100200090012000244FF4BA
:2009C0008029DFF8748003902AE000BFFFF786FED8F8001006EBC420CA4313041B0C12D0EB
:2009E0000B049B0903F1006383420ED9A0F10060C00A02900120019004A9684600F020FBDC
:200A000060B100270EE04B46ECE71204120C03D009048909401AE9E74946FBE7641CA4B235
:200A2000AC42D3D300F078FB3846B3E7FFFF0F080030000800200240E075FF1F0048704786
:200A40000030000803494FF0FF30086001F50171086070471001002010B5CA0501D00020FF
:200A600010BD02688A4204D002C04FF40072FFF73FFE012010BD000070B504460C480D46F1
:200A8000844202D1A0F501740AE00A48854202D1074C054604E0204600F034F8002806D0DB
:200AA00029462046FFF7D8FF002800D0204670BD140300200030000830B40E4B1C1A4B1EBE
:200AC0009C4207D30C4B984204D34418641EB4F1016F02D330BC00207047440A64029C4239
:200AE0000B46014601D1054800E0054830BCFFF7E7BE0000FFFF0F08003000081403002007
:200B0000100100202DE9F04707464FF0010800F05FFB14494FF4004008610024386800EB80
:200B2000C40907EBC40045688668FFF7D7FD2A4633464946002000F0F9FA10B14FF000084A
:200B40000AE0D9F80000D9F80410684071400843F4D1641C402CE1D300F0DEFA4046BDE8F9
:200B6000F087000000200240018840884AF25A52514040BA4840704710B5044601202080C9
:200B80000020A070E0702046FFF7EEFFA08010BD70B5114801684068CA4372EA000215D0C0
:200BA0008BB20C0C0D4A44EA0044090E1380947041EA0021D17090801446B3F5006F05D284
:200BC0001046FFF7D1FFA188884202D00348FFF7D3FF024870BD000000F803085C0000202B
:200BE000F0B590F820500468A468012D05D0022D03D0416A41F480214DE014F0406F01D1A8
:200C0000E50045D5C4F301640125A5401D608D684FF4C0739DB1CE6835434E6845EAC6051A
:200C2000066803EB0417F5514FF4C275076805EB04150E697E51097D012905D009E00E88BB
:200C4000CD6845EA4655EBE701684E5946F480764E511179D2F805504FF4C67641EA05216B
:200C6000056806EB0416A9511178D2F801204FF4C47541EA0221026805EB04155151006847
:200C800003EB0411425842F0010242500020F0BD416A41F4001141620120F0BD10B590F874
:200CA0002020012A07D0022A05D0416A41F480214162012010BD0068D0F8002242F0010258
:200CC000C0F800220A7D02F01F0301229A40D0F81C329343C0F81C32CB69B3B9D0F80C320A
:200CE0009343C0F80C328C894B6864F31F434C6900EBC404C4F840320C890B6864F31F4350
:200D00004C6900EBC404C4F84432CB69012B16D1D0F80C321343C0F80C320C884B6864F302
:200D20001F434C6900EBC404C4F840320C89CB6864F31F434C6900EBC404C4F844328B69AC
:200D4000002BD0F804320FD053EA0203C0F804320B69002BD0F8143208D01343C0F8143282
:200D6000096A012904D008E09343EFE79343F5E7D0F81C121143C0F81C12D0F8001221F0A1
:200D80000101C0F80012002010BD70B590F82040012C05D0022C03D0416A41F4802128E001
:200DA000046809B32469A40720D04FF4D874056804EB01142D5915F00405956005682D5967
:200DC0001AD0ED08556005682C5904F00204D4604FF4DA74056804EB01142E5906F00F06CB
:200DE000082E0CD308250DE0E468DCE7416A41F400114162012070BD6D0D1560E3E72D5994
:200E000005F00F05156105682D59C5F30725956105682C59240C54614FF4DC72046802EBC5
:200E20000112A4581C700468A458240A5C700468A458240C9C700468A258120EDA704FF4FE
:200E4000DE72046802EB0112A4581C710468A458240A5C710468A458240C9C710468A258DF
:200E6000120EDA71006829B1016941F020010161002070BDC16841F02001C160F8E770B5BA
:200E8000040003D094F8200010B104E0012070BD204600F090F82068016841F00101016079
:200EA00000F0AAF90546052604E000F0A5F9401B0A2811D820684068C007F6D02068016893
:200EC00021F00201016000F097F905460BE000F093F9401B0A2806D9606A40F4003060620F
:200EE00084F82060D2E7206840688007EFD4207E0128206801683DD021F080010160607E2D
:200F000001282068016838D021F040010160A07E01282068016833D021F020010160E07ED0
:200F20000128206801682ED041F010010160207F01282068016829D021F008010160607FEA
:200F400001282068016824D021F004010160D4E902010843D4E90412114308436168491E5F
:200F600008432168C86100206062012084F82000002070BD41F08001C0E741F04001C5E711
:200F800041F02001CAE721F01001CFE741F00801D4E741F00401D9E70346002093F8202057
:200FA000012A01D0022A05D11A6889069268914300D001207047704770B5044690F82000DE
:200FC000012804D0606A40F40020606218E0022084F820002068016821F00101016000F029
:200FE0000BF905460EE000BF00F006F9401B0A2808D9606A40F400306062052084F82000E7
:20100000012070BD20684068C007EDD1606270BD0A4810B54FF0FF318163C1630022826349
:20102000C2630164026481628262C162C2620163026300F015F9002010BD000000100240AC
:201040002DE9F05F054632488946017801290CD00126804606704CF2503B5846FFF7FEFB5F
:2010600007004FF0000A03D04EE00220BDE8F09F51464046C8F804A0264C226892050AD5D6
:201080002168490505D5216821F480612160032109E0067708E02268520504D5216821F4D5
:2010A00080612160022101772868012807D04FF0FF31C9F8001040F2FA3BAE681DE0686819
:2010C000FFF786FB5846FFF7C9FB0746606920F00400606116E030466968FFF787FB4CF263
:2010E0005030FFF7BBFB0700606920EA0B00606102D0C9F8006005E0761CD5E902010844A7
:20110000B042E8D8FFF736FB88F800A03846ADE714000020002002400348416941F00041C7
:201120004161002070470000002002402DE9FF5F254C0646904620789A4601280BD0012030
:2011400020704CF2503B5846FFF788FB07004FF0000904D02AE0022004B0BDE8F09F48465A
:20116000C4F80490194D2968490504D5286820F4806028600220207726B1012E09D0022E2D
:2011800007D00CE0424653460198FFF743FB012612E041460198FFF74BFB022E0AD0584681
:2011A000FFF75CFB4FEA0007FFF7E4FA84F800903846D1E74FF480265846FFF74FFB074678
:2011C0006869B0436861EFE71400002000200240064900204A69002A07DA054A8A60054A61
:2011E0008A604969002900DA012070470020024023016745AB89EFCD00F088BD10B5002438
:20120000032000F0CBF80F2000F008F808B1012401E000F059F8204610BD000070B50E4E25
:2012200005460024307898B14FF47A71B1FBF0F00A490968B1FBF0F000F0C2F840B9102D64
:2012400006D200222946501E00F088F8756000E00124204670BD000008000020340000205E
:2012600010B500F0D3F94FF090442020A062134800F0EEF8124800F0EBF8204600F0E8F804
:201280001048816D21F000718165016E21F480410166C16C21F00401C164C16C21F002014B
:2012A000C164C16C21F00101C164816D21F080518165016E21F00101016610BD00080048E8
:2012C0000004004800100240F0B587B0012000F0B3F84FF0805000F0A3F8012000F084F8B1
:2012E000022000F081F8042000F07EF84FF4804000F0A2F84FF0007000F092F84FF400469A
:20130000012000240096CDE90104CDE903404FF090456946284600F0DDF8AE614FF4C060D6
:201320000226CDE9000607200327CDE90440CDE902746946284600F0CDF83802CDE900068A
:201340000920CDE90440CDE902746946024800F0C1F807B0F0BD000000040048F0B40E4BEF
:201360001B680C46C3F30223C3F10705042D00D90425191D072901D2002300E0DB1E01266E
:2013800006FA05F1491E214099409E40761E16403143F0BC00F0DCBE0CED00E0064900F02C
:2013A000070208684FF6FF03184040EA0220034A10430860704700000CED00E00000FA0532
:2013C00010B5401EB0F1807F01D3012010BD4FF0E02460610F21601700F0BAFE0020A06114
:2013E00007202061002010BD044908B5CA6C0243CA64C96C0140009108BD00000010024087
:201400000249CA6A0243CA6270470000001002400249CA6A8243CA6270470000001002405A
:20142000044908B58A6D02438A65896D0140009108BD000000100240044908B50A6E0243D1
:201440000A66096E0140009108BD00000010024010B50024B0F1904F07D01949884209D176
:201460000220FFF7CDFF022023E00120FFF7C8FF01201EE01349884204D10420FFF7C0FF92
:20148000042016E01049884204D10820FFF7B8FF08200EE00D49884204D11020FFF7B0FF85
:2014A000102006E00A49884206D18020FFF7A8FF8020FFF7ADFF00E00124204610BD00006B
:2014C0000004004800080048000C004800100048001C0048F0B50A680F2692FAA2F2B2FA48
:2014E00082F303248AE001259D402A407ED04D68012D01D0022D20D18D68876892FAA2FC49
:20150000BCFA8CFC4FEA4C0E04FA0EFC27EA0C0792FAA2FCBCFA8CFC4FEA4C0C05FA0CF5D5
:201520002F438760CF680D68D0F804C02CEA050C7D434CEA050CC0F804C00F69D0F80CC064
:2015400092FAA2F5B5FA85F54FEA450E04FA0EF52CEA050C92FAA2F5B5FA85F56D00AF40E3
:201560004CEA070CC0F80CC04D68022D2FD1FF2A15D8D1F814C0056A92FAA2F7B7FA87F744
:20158000BF0006FA07F7BD4392FAA2F7B7FA87F7BF000CFA07FC45EA0C05056217E0D1F80B
:2015A00014E0476A150A95FAA5FCBCFA8CFC4FEA8C0C06FA0CFC95FAA5F5B5FA85F5AD0021
:2015C00027EA0C070EFA05FE47EA0E0747624D68076892FAA2FCBCFA8CFC4FEA4C0C04FAD2
:2015E0000CFE27EA0E0792FAA2F200E005E0B2FA82F2520095402F4307605B1C0A6832FAA1
:2016000003F57FF470AF0020F0BD00001E4808B5016841F0010101600168C1F340010029CC
:20162000FAD0016821F0F00141F060010160416821F47F414160416821F0F85141F080515E
:201640004160002181600268104B1A4022F0806200920260026812F0206FFBD14FF4805204
:20166000C2600261026822F480220260816140F27F7100910162D0F8941041F40001C0F80F
:201680009410002008BD000000100240FFF4FEFE10B5044600F092F9206000F065F9606068
:2016A00000F070F9A060606800F07AF9E06010BD70B500242F49304D4FF40046032804D0D3
:2016C0000C281ED0302837D034E0D1F8880000F0030040F44030B0F5403F0BD06FF44031BA
:2016E000401804D001283ED0022823D135E000F065F91EE000F062F900F036F900F050F965
:2017000017E0D1F8880000F00C0040F44020B0F5402F08D0001FB0F54020E8D0042822D00B
:20172000082807D119E000F049F900F01DF900F029F90446204670BDD1F8880000F0300010
:2017400040F44010B0F5401FEDD01038B0F54010CDD0102807D02028ECD100F017F800282F
:20176000E8D03446E6E700F009F80028E2D02C46E0E70000001002400024F400024800684A
:20178000C0F3802070470000001002400248D0F89000C0F34000704700100240024800689D
:2017A00000F0F00070470000001002400248D0F8940000F47060704700100240024800681B
:2017C000C0F3C00070470000001002400248C06800F0700070470000001002400248C06840
:2017E00000F00300704700000010024001490860704700003400002070B5044600680D4606
:20180000012610F0010F35D1E9686868AA69084329691143084321681E4A114008432060CE
:20182000A868616821F44051014361606869A16821F440710143A1601748844201D1032025
:2018400008E01648844201D10C2003E01448844210D13020FFF72CFF60B1296851B1AA6970
:201860000026B2F5004F07D000EB5100B0FBF1F080B2E060304670BD400000EB5100B0FB71
:20188000F1F081B24FF6F07201EA0200C1F342010843EEE7F369FFEF003801400044004042
:2018A000004800404FF090414FF40040886270472DE9F04710490026354648804FF40044D6
:2018C0004FF090484FF496790C4F07E066B10026C8F82840484600F04BFC6D1C3868008882
:2018E000A842F3DCBDE8F0870126C8F81840C82000F03EFCF2E70000000000204400002065
:2019000010B500F003FA0B4C616888420DD322784FF400404FF0904142B10022227088628D
:2019200000F0F4F961880844606010BD012222708861F5E70000002010B500F013F8002886
:2019400003D0BDE81040FEF7F7BF10BDFFF70EB8FFF774B8FFF776B8AFF30080012070474B
:20196000FFF7AAB80120704704498968044A01F0F0010909515CC8407047000000100240F9
:20198000A821000804498968044A01F4E06102EB11210978C840704700100240E8210008F2
:2019A00004498968044A01F4605102EBD1210978C840704700100240E8210008184810B54E
:2019C0008068184C10F00C0005D004281AD008281AD00C281AD0FFF7F1FED8B1FFF7EEFE3C
:2019E00050B1FFF7DBFE09E0FFF7D8FE02E000BFFFF7DCFE000A02E0FFF7D8FE000954F8E4
:201A0000200010BD084810BD084810BDBDE8104000F00EB8FFF7D2FE0028E9D0E4E7000082
:201A200000100240B82100080024F40000366E0110B5FFF7D3FE1D4C012803D002282AD0A1
:201A400003282AD0FFF7BAFE28B1FFF7B7FE48B3FFF7A4FE06E0FFF7B1FE00B3FFF79EFECC
:201A6000000A00E0000954F8204000BFFFF7AEFE012101EB1010B4FBF0F20D48C368C068FF
:201A8000C3F306235A4300F0C06001EB50604000B2FBF0F010BD074CE8E7074CE6E7FFF74C
:201AA00085FEDDE7FFF782FEDCE70000B8210008001002400024F40000366E0110B588B0B9
:201AC0001C216846FEF7D2FB104C206820F0010020604FF4E1300090002001900C21029090
:201AE000CDE903010590069069462046FFF784FE606820F490406060A06820F02A00A060C6
:201B0000206840F00100206008B010BD00380140054A01460020D369C3F34013002B02D096
:201B2000506A087001207047003801402DE9F0411C4C80461C4D60780F46002680B1207828
:201B40002844401CFFF7E4FF012819D000F0DEF86168C831884200D966700020BDE8F0819B
:201B60001148FFF7D5FF0128F7D12878401E8028F3D800F0CBF86060267001206070ECE713
:201B80002078401CC2B2227028789042E5D12270691C4046FEF7ACFD6670207838700120B1
:201BA000DCE700004C0000201805002070B5094DA86200F0ABF800F10A0405E0FEF78EFD3D
:201BC00000F0A4F8A04204D8E869C0F3C0100028F4D070BD0038014070B50D4606468129E7
:201BE00003D9982108A0FEF7A2FB2846FFF7DEFF002406E0FEF772FD305DFFF7D7FF641C8E
:201C0000A4B2AC42F6D370BD2E2E5C447269766572735C4F70656E424C545C72733233324B
:201C20002E630000704700002A4810B5016821F0070141F004010160006800F00700042881
:201C400003D06A2124A0FEF772FB2848016821F4C06141F4007101602548016841F48071EE
:201C600001600168C1F380210029FAD0416821F0F85141F080514160C26840F602211D4BC1
:201C80001A401143C160C16841F08071C160016841F0807101600168C1F340610029FAD06C
:201CA000816841F003018160816801F00C010C29FAD1816821F0F0018160816821F4E06133
:201CC0008160816821F460518160BDE810400A48FFF78CBD002002402E2E2F436F72652F68
:201CE0005372632F6D61696E2E63000000700040001002408C80FFF900B4C4040248016822
:201D000041F470010160704788ED00E000B500F05DF80148406800BD54000020184808B577
:201D2000816D41F001018165816D01F0010100918168144A01F4E06102EB112180680A7824
:201D400011490968D14010F4E06F16D0022041430122900702604FF6FF72C2620B4AB1FBD1
:201D6000F2F1491E8162416941F001014161084900224A60406A088008BD0120E7E70000B4
:201D800000100240E821000834000020A0860100540000200B48816B41F001018163816BAF
:201DA00021F001018163816D21F0010181654FF0E020002101614161816103494FF0007004
:201DC000086070470010024004ED00E04FF08040416A0A480288891A89B264290CD364236A
:201DE000B1FBF3F143680B44436001EBC10303EB011102EB810101807047000054000020EB
:201E00002DE9F041114FFF21001D397000F092F804460025D7F8886006E000BF16F8010BD6
:201E20002844C5B2FEF75AFC641EF7D20121797028463C46391D00F083F90020A070E070EC
:201E40000820A4F88600BDE8F08100009C05002070B50F4C0020012584F8820084F8815050
:201E6000FF21217010216170A070FEF7BFFBE070FEF7CCFB2071FEF7C9FB000A6071A571A9
:201E8000E5710820A4F88600BDE87040FFF762BD9C05002070B50446FEF7A8FB6178801EF9
:201EA000884201DA222018E00E4DFF2028700120A5F88600617859B1A21CD5F88800FFF701
:201EC0004FFD48B155F8880F61780844286070BDFFF732FD0028FAD13120BDE8704000F051
:201EE00025B900009C05002070B50546FEF77EFB6978401E884204DABDE87040222000F0F7
:201F000015B9281D00F016F8094C0146C4F888006A78601CFEF7ECFBFF2004F8480B697847
:201F2000206C084420646878401CE08770BD00009C0500200178427841EA02218278C07801
:201F400041EA024141EA0060704700000548002100F8811FC0F80710C170A0F8051081702D
:201F6000417070479C050020034890F88100002800D00120704700009C0500202DE9F0410C
:201F800001780127634C0546FF2912D094F8810001287AD10020FF26F32941D011DCD029C3
:201FA00078D009DCC9295DD0CC2970D0CF296FD196E0FFF74DFF8EE0D1297BD0D22967D1CA
:201FC0006CE0F4390B2963D2DFE801F02106259090902E903B3D4700FEF708FB6A78401EB6
:201FE000904201DA222071E0601CD4F888104834FEF77EFB04F8486D6978D4F888000844A5
:20200000C4F888006878401CA4F8860063E02846FFF76AFF5FE02670281DFFF78BFF31E063
:202020002846FFF7EDFE56E026703B49C4F888106070A070E0700720211D00F081F8082087
:20204000E2E7002042E02670607094F88210A170E070207160710620D6E784F8810084F8D2
:2020600082003FE0FEF7C2FA411E6A1CD4F88800FFF776FC58B12670FEF7B8FAD4F88810C3
:20208000401E0844C4F8880023E041E002E02BE02CE00FE02846FFF7FDFE1CE02670607085
:2020A0000546A070FEF7A2FAE07025716571A5710720A9E72846001DD4F88850FFF73AFF4D
:2020C00001462846FFF742FC70B10BE000F02EF801E0A4F8867094F88400012808D00AE087
:2020E000FEF716FB2670F4E73120EFE72020EDE7102000F01BF8B4F98600002808DD84F83F
:202100008470BDE8F041034A81B21046FEF7C8BABDE8F0819C050020142200080249002028
:2021200081F88400704700009C0500200349FE220A7048700220A1F8860070479C050020D3
:202140000870020A4A70020C8A70000EC87070470907090E002804DB00F1E02080F8001491
:20216000704700F00F0000F1E02080F8141D704730B50446FFF7CAFD0546601C00D0641C55
:20218000FFF7C4FD401BA042FAD330BDFFF736F8FFF74AFDFEF702F9FEF716F9FCE74FF01A
:2021A0004070E1EE100A704700000000000000000102030406070809A0860100400D030030
:2021C000801A060000350C0040420F0080841E0000093D0000127A000024F40000366E01DC
:2021E0000048E801006CDC02000000000102030405020602060307030803090309040A0406
:202200000B040C040C050D050E050F050F061006100710084F70656E424C54003C22000821
:202220000000002064000000C8010008A022000864000020240C0000E401000800000000DE
:2022400000000000010000001000000000000000000000000000000000000000000000006D
:202260000100000000000000000000000000000000093D0000000000000000000000000017
:20228000000000000500000000000000000000000000000000000000000000000000000039
:20300000B8080020D9320008137D000893780008117D0008A153000855870008000000009C
:20302000000000000000000000000000C17E0008EB53000800000000157D0008C37E000820
:20304000F3320008F3320008F3320008F3320008F3320008F3320008F3320008F332000808
:20306000F3320008F3320008F3320008F3320008F3320008F3320008F3320008B153000809
:20308000F3320008F3320008F3320008F3320008A5530008F3320008F3320008F3320008F5
:2030A000F3320008F3320008F3320008F3320008F33200080000000000000000F332000802
:2030C000F3320008F3320008F3320008F3320008F33200083D870008F3320008F3320008E9
:2030E000F3320008F332000800000000000000000000000000000000000000000000000076
:2031000000000000F332000800000000F33200080000000000000000F3320008F3320008FB
:20312000F3320008F3320008F3320008F3320008F3320008000000000000000000000000AE
:20314000F3320008F3320008F332000800000000F3320008F3320008F3320008F332000834
:20316000F3320008F3320008F332000800000000F3320008F332000800000000000000006E
:20318000F3320008F3320008F332000800F002F800F092F80AA090E8000C82448344AAF1EE
:2031A0000107DA4501D100F087F8AFF2090EBAE80F0013F0010F18BFFB1A43F001031847A9
:2031C000905C0000B05C0000103A24BF78C878C1FAD8520724BF30C830C144BF04680C607F
:2031E000704700000023002400250026103A28BF78C1FBD8520728BF30C148BF0B607047EF
:203200006E2900F01583702900F05F84662905F07985652905F07685672905F0738561291C
:2032200005F0728503681B0A28BF41F08001692900F0C282642900F0BF82752900F0BC8229
:203240006F2900F0ED83782900F02B84E92900F08783E42900F08483F52900F08183EF29FC
:2032600000F0EA83F82900F02A840368DB0928BF41F08001632901F07781732901F07C814B
:20328000E32901F08781F32901F08C81002070471FB505F032FD01F091FB0400002000217E
:2032A00005F09EFC401C60600020002105F082FCE0601FBD10B510BD01F052FB1146FFF776
:2032C000E7FF05F03FFB01F02BFC03B4FFF7F2FF03BC01F06FFC0000094880470948004758
:2032E000FEE7FEE7FEE7FEE7FEE7FEE7FEE7FEE7FEE7FEE704480549054A064B70470000EB
:20330000357F00088D310008B8020020B8080020B8040020B804002053EA020C00F0698095
:203320002DE9F04B4FF00006002B1FBFB3FA83F503FA05F424FA05F65E4012BF1643B2FA46
:2033400082F502FA05F4C5F120051EBF22FA05FC44EA0C04203556EA044C4FEA144418BFA1
:20336000641C4FF000084FF00009904271EB030C39D3002919BFB1FA81F701FA07F6B0FA2F
:2033800080F700FA07F6C7F120071EBF20FA07FC46EA0C062037B6FBF4FCA7EB0507103FBF
:2033A00007F01F0BCBF120060CFA0BFB2CFA06F644BFB3460026202FA4BF5E464FF0000B1A
:2033C0005BEA060C08BF4FF0010B19EB0B09ABFB027C48EB0608C01B06FB02CC0BFB03CC88
:2033E00071EB0C01C1E70B46024641464846BDE8F08B13B54FF000004FF00001AFF3008085
:20340000BDE81C40704700007CB51D4616460C00009001D02044401E074B7B442A466946A5
:203420000190304600F01DFA05461CB10020694600F02AFA28467CBD750400000FB400B5EB
:203440008DB010A9099000910B904FF0FF300A9000200C90064878440690064878446A4693
:2034600007900F9909A800F013FC0DB05DF814FB570800006F0800002DE9FF5F1D464FF050
:20348000FF3B91464FF000085F46D5E90146A96901987F1C8847296A824688470028F6D1FC
:2034A000BAF1FF3F0CD0002E24F4C06419DD600614D5BAF12B0F09D0BAF12D0F0ED103E031
:2034C000584604B0BDE8F09F44F48064A96901987F1C8847761E8246002E02DDBAF1300FE2
:2034E00003D0B9F1000F26D032E0A969761E01987F1C44F400748847002E824605DDBAF160
:20350000780F06D0BAF1580F03D0B9F1000F10D01EE0B9F1000F02D0B9F1100F18D1A96983
:20352000761E01987F1C24F4007488478246102002E0082000E00A20814609E0A96908FB97
:203540000908761E01987F1C44F4007488478246002E05DD4946504600F086FB0028EDDABA
:20356000E96901988847A00502D46FF00100A8E7E00725D1600613D5600502D5C8F1000007
:2035800000E0404629680A1D2A600968220501D5087015E0220701D5088011E008600FE0D9
:2035A0002868011D29600068210502D580F8008006E0210702D5A0F8008001E0C0F8008061
:2035C00038467EE740EA010370B59B072ED14FF00136042A2AD308C810C99D1B9D43121F01
:2035E00015EAC61517D0D8B2E1B2401A50EA056110D198B2A1B2401A50EA05410AD123F0AD
:203600007F4024F07F41401A50EA052102D1180EA0EB146070BDA342DBD018BA21BA884231
:2036200001D9012070BD4FF0FF3070BD0AB9002070BD10F8013B11F8014B63B1A3420AD14A
:20364000521E08D010F8013B11F8014B1BB1A34201D1521EEDD1181B70BD4FF0000204290A
:20366000C0F0128010F0030C00F01B80CCF1040CBCF1020F18BF00F8012BA8BF20F8022B3C
:20368000A1EB0C0100F00DB85FEAC17C24BF00F8012B00F8012B48BF00F8012B70474FF00A
:2036A000000200B5134694469646203922BFA0E80C50A0E80C50B1F12001BFF4F7AF090716
:2036C00028BFA0E80C5048BF0CC05DF804EB890028BF40F8042B08BF704748BF20F8022B67
:2036E00011F0804F18BF00F8012B704770477047704770B5044685690068C10601D530266B
:2037000000E02026C00707D070BDD4E9012130469047206A401C20626D1EF6D570BD70B57C
:20372000044685690078C00707D170BDD4E9012120209047206A401C20626D1EF6D570BD2C
:2037400009684A0501D540B27047C905FCD500B2704709684A0501D5C0B27047C905FCD5C4
:2037600080B2704770B50C460546012A05D02878800600D5EA69002302E0012305E05B1CCB
:20378000934202D2E05C0028F9D1A869E618C01AA861286A184428622846FFF7AAFF04E0F7
:2037A000D5E9012114F8010B9047B442F8D32846FFF7B5FF70BD00002DE9F041064600247D
:2037C00010687529314616A510D0FFF7B9FF002802DA404213A507E031688A0701D512A537
:2037E00002E0490704D511A5012401E0FFF7B1FF00210A2206F1240709E0B0FBF2FCB0FBC0
:20380000F2F302FB1C00303078541846491C0028F3D123462A463046BDE8F04100F0B6BA4A
:20382000000000002D0000002B0000002000000011680268006A530501D508700AE0D3055B
:2038400001D5088006E0130603D5C217C1E9000200E008600120704701694A1C02610878DB
:20386000704700B58FB0CDE901310021059105497944CDE903101146684600F031F90FB04C
:2038800000BD0000E5FFFFFF0A6802F8010B0A607047D1E900239A4202D2531C0B60107009
:2038A000704700002DE9FF5F15468A460446DFF8AC80F8440027D8E900103E46CDE90010E7
:2038C00010E03AF816106A4602A801F029F8411C07D02178890603D5E269391891420DD8AC
:2038E0000744761C2078800602D5E069B84205DDAE42E6DB3AF816000028E2D1A069C01B19
:20390000A0612046FFF7F5FED8E90010CDE90010002017E03AF818106A4602A801F000F80C
:20392000B0F1FF3F81460BD000250DF1080B05E0D4E901211BF8050090476D1C4D45F7D338
:2039400008F10100B0428046E4DB206A384420622046FFF7E4FEBDE8FF9F00009E540000FB
:203960002DE9F0418046D21D22F007020025D2E90002F52915A614D0011E72F1000106DA2E
:203980000023D0EB030063EB020211A608E0D8F800108B0701D50FA602E0490701D50EA69C
:2039A00001251146002408F1240704E000F0A0F930323A55641C50EA0102F7D12B46324676
:2039C00021464046BDE8F04100F0E0B9000000002D0000002B0000002000000030B400211E
:2039E00000F1240408E002F00705D208303542EA4372DB086554491C52EA0305F3D1046833
:203A0000002310A2250708D504F020040C4304D0C46901230CA2641EC46130BC00F0B6B99C
:203A200010B5044621461068FFF793FE02462046BDE810400023D1E7D21D22F00701D1E9D0
:203A40000023CBE70000000030000000F0B40D460188090502D5214C7C4402E01F4C7C44C2
:203A60000E34002100F1240608E002F00F071209E75D42EA03721B097754491C52EA03073E
:203A8000F3D102780023120704D5702D06D009B1022311342246F0BC00F078B9012310349F
:203AA000F8E770B504460D4621461068FFF751FE024629462046BDE870400023C6E7D21D10
:203AC00022F00703D3E90023C0E70368126843F0200303600823C3610023B7E70053000043
:203AE0002DE9F05F894604464FF0000ADFF874B1FB44C0F820A02046E1688847002874D062
:203B0000252806D0D4E901219047206A401C2062F1E700265F462046E168884720280546B0
:203B200007DB312D05D2781910F8200C08B10643F1E7B00701D526F00406C4F81CA0002783
:203B4000C4F818A02A2D09D0284604F043FE38B304EB8708303DC8F8185019E059F8041BB7
:203B6000204604EB87029161E1688847012F054618D1E069002820DA26F020061DE0D8F885
:203B8000180000EB800005EB40003038C8F818002046E1688847054604F01CFE0028EED174
:203BA000012F0AD02E2D08D12046E16888477F1C0546022F46F02006C4DBA069002803DA29
:203BC000404246F00106A061F00701D026F010066C2D0BD0682D09D04C2D39D06A2D35D031
:203BE000742D35D07A2D33D016E038E0E1682F4620468847B842054609D16C2F26D04FF481
:203C00008060E168064320468847054604E06C2F1AD04FF4807006430DB3A5F141001928F5
:203C200002D8203546F400664A462946204626604E46FFF7E5FA80B101280BD0F61D26F003
:203C4000070000F1080956E74020E4E78020D8E70020D6E706F104094DE7284652E7206A4E
:203C6000BDE8F09F905200003A2800D2303820F02002412A01D3A2F13700884201D34FF07A
:203C8000FF307047026811441378016018467047D1600549794451610449794411620021F2
:203CA0001161114600F082BCEDFFFFFFDD000000426842B1016811F8013B23B1521EC0E90E
:203CC0000012184670470121C160881E704742685AB1C368016843B983688B4205D0491EE4
:203CE000521CC0E90012002070474FF0FF30704730B5B0F10A024FEA900E71F100034EEA99
:203D0000817EB0EB0E0061EB91014FEA101E4EEA017E10EB0E0041EB11114FEA102E4EEAF9
:203D2000016E10EB0E0041EB11214FEA104E4EEA014E10EB0E0041EB1141401841F100017D
:203D40004FEAD00040EA41704FEAD10110EB80054FEA810444EA907444EB01046D1944EB1B
:203D60000404521BA3414FF0000348BF0A3200D530BD401C41F1000130BD10B5044600F028
:203D800015FE0068005D00F0010010BD2DE9F0470D4699469246044600F1240801688806D8
:203DA00004D5E06921F01001216000E00120A84201DD471B00E00027A1697A1902EB090079
:203DC000081AA0612078C00602D42046FFF791FC002608E0D4E901211AF806009047206A3D
:203DE000401C761C20624E45F4DB2078C0060AD52046FFF77EFC06E0D4E9012130209047F2
:203E0000206A401C2062381EA7F10107F4DC07E0D4E9012118F805009047206A401C20625A
:203E2000281EA5F10105F3DC2046FFF778FC2078000602D50220BDE8F0870120FBE7704794
:203E40002DE9FF4F0C461E464FF0FF378BB0D2E90001DDF860800A908A46C1F30A5505B9EC
:203E60003D46002108464FF00000BAF1000F00F4400005DA00EB80004FF4400101EA50001A
:203E80004FEA9059B9F1010F00DDB9460A9850EA4A000ED044F61050A5F2FF3545432F1436
:203EA000B8F1000F1ED07542291E1EDDC9F100021CE0B8F1010F4FF0000001D0302103E0AE
:203EC000F24305E02154401CB042FBDB30460022002121540B99C1F80880C1E900200FB093
:203EE000BDE8F08FBD1B6D1CDEE74A4600DA694206A800F0A7FD06AB93E8070003AB83E8D5
:203F0000070050460A9900F05CFE8DE80700A0F500501F3800900398002D09DD42F21F01CD
:203F20004A46084403A90390684601F0BBF808E0A0F500504A461F3803A90390684601F082
:203F4000C5F88DE807000004000C03D04FF0FF30410800E01046B8F1000F03D00022009219
:203F600015461EE0751E05D4FFF7C2FE303262556D1EF9D5B3460122084302D000227F1C5E
:203F800004E02078302801D100227F1E002A099786D01DE0112D07DAFFF7AAFE30326255C9
:203FA0006D1C50EA0102F5D1084302D00098C8B10EE00021681E05E0235C625C6354225463
:203FC000401E491C8142F7DBAB46A81B401E0990002004F80B000B98099AC0F80880C0E988
:203FE000002B7CE711264FF0000859E72DE9F04F88460446D21D22F0070191B0D1E9000103
:20400000CDE90A0104F0A7FB02460B98C00F01D02D2007E02068810701D52B2002E0202136
:2040200001EAC000032A099001D0072A05DB03464146204600F0C6FC0BE12078800601D565
:20404000E06900E00620B8F1650F814606D0B8F1660F18D0B8F1670F70D131E00020B9F116
:20406000110F009001DB112301E009F101030AAA01A90CA8FFF7E4FEDDE90C70002609F155
:204080000105834647E001204B4600904FF000470AAA01A90CA8FFF7D3FEDDE90DB00C9961
:2040A0005D46002610B909F101000D18B9EB050003D4C0F1FF3609F10105A5EB09002BE044
:2040C000B9F1010F01DA4FF001090020B9F1110F0090484601DD112300E003460AAA01A961
:2040E0000CA8FFF7ADFEDDE90C704D4600268346207800070AD4AB4500DA5D4601A8012DE6
:2041000004DD411911F8011C302907D04F4502DA17F1040F04DA012082460FE06D1EEEE76D
:20412000002F02DCED1B3E4403E0781CA84200DD7D1CB81B00F1010A4FF00047207800071D
:2041400003D4AA4501DB4FF0FF3A0021B7F1004F0DF143088DF8431024D002202B23002F79
:2041600001DA7F422D230A21021EA0F1010000DC5FB197FBF1FC97FBF1F201FB1C7C1746A5
:204180000CF1300C08F801CDEEE7A8F1010003702188090501D5452100E06521A0F1010843
:2041A00000F8011C09980FA9A1EB0807FF1D00B10120411901EBEA70A1693844081A401E62
:2041C000A0612078C00602D42046FFF792FA099828B1D4E901219047206A401C2062207892
:2041E000C00622D52046FFF784FA1EE0002E04DBB34502DD01A8805D00E03020D4E90121B1
:204200009047206A401C2062761CAAF101005FEA000A0AD100F0D2FBC0680168405CD4E95C
:2042200001219047206A401C2062281EA5F10105DCDC07E0D4E9012118F8010B9047206A40
:20424000401C2062381EA7F10107F3DC2046FFF766FA032011B043E62DE9F04F04460D4600
:20426000D21D22F0070089B0D0E9009248461746394604F070FA0246F80F01D02D2307E093
:204280002068810701D52B2302E0202101EAC0038DF820300BB1012000E00020032A824672
:2042A00001D0072A04DB2946204600F08BFB3DE12078800601D40D2500E0E569C7F30A5647
:2042C0000D2D49DA00214FEA175B08464FF00000002F00F4400007DA00EB80004FF44001F5
:2042E00000EBD07001EA60008115012901DD4FF0FF3100224FEA850CBCF1180F06D3134649
:20430000ACF118004FF08052C24003E04FF4801323FA0CF30CF10C0CBCF1200F04D3ACF19B
:20432000200C09FA0CF001E007FA0CF000294FF0004801DD18B90FE00ED140450CD319EBDF
:2043400002095F4121B9404502D19F4329EA0209BBEB175F00D0761C2088000502D57B48BB
:20436000784402E079487844193808AA302302F80A30037C0AF10101002E0AF1020A535440
:204380006A4602DC4FF0300101E04FF031014FF001088DF8001002D0A6F2FF3603E059EA2B
:2043A000470100D06A4E002D02DC2178090704D54FF002082E218DF80110C44600210BE05C
:2043C000C7F303433F01C35C491C6D1E02F80830052908F1010801DA002DF1DC00210CE04A
:2043E00000EB1973491C1B786D1E082902F808304FEA091908F1010801DA002DF0DC217896
:20440000890602D514E0A8F10108E04505DD02EB080111F8011C3029F5D0B8F1000F07DDC3
:2044200002EB080111F8011C2E2901D1A8F10108002D05DD3E2102F808106D1E08F1010888
:20444000407C002E02F8080008F1010804DA2D20764202F8080002E02B2002F808000A212F
:204460004FF47A70864208F101080BDB96FBF0F3303302F8083096FBF0F308F1010800FBE5
:20448000136601E0642E0CDB642096FBF0F3303302F8083096FBF0F308F1010800FB1366D2
:2044A00001E00A2E06DB96FBF1F0303002F8080008F1010896FBF1F001FB1060303002F8F4
:2044C0000800A16908F1010808EB050202EB0A00081AA0612078C00602D42046FFF709F922
:2044E000216A08AE01EB0A00206204E0D4E9012116F8010B9047BAF1010AF7D22078C00672
:2045000002D52046FFF7F5F86E4609E016F8010B3E280FD0D4E901219047206A401C206261
:20452000B8F10108F2D22046FFF7F9F809B00320BDE8F08F206A2844206203E0D4E901217E
:20454000302090476D1EEBD3F8E70000444A000002FCFFFF10B5436913B1AFF3008001E04A
:20456000FFF700F9012010BD127800F124010A7000224A700122EDE711684FF0FF32E9E7B8
:2045800010B5436913B1AFF3008001E0FFF78AF9012010BD128800F1240182840022C2845E
:2045A0000122EDE711684FF0FF32E9E72DE9F34F4FF0000A0C4656468DB001200C9001F1D0
:2045C0000C000B9062690B980121904705002DD0252D2CD0216A8847C0B162690B98012122
:2045E0009047216A88470028F7D16269411E0B98904700E0761CA1690D988847216A8847AC
:204600000028F7D1E1690D988847DBE7A1690D988847A842074601D1761CD3E7E1690D9868
:2046200088477F1C02D1BAF1000F6FD06BE162690B9800273D46394690472A2804D1626998
:204640000B98012190470125DFF8D08262690B9801219047A0F130010A290AD24745E5DCEA
:2046600007EB870100EB4107303FDFD445F01005ECE7E90601D46FF000476C280AD04C2802
:2046800014D0682815D06A280DD074281CD07A281AD01DE062690B98012190476C2802D074
:2046A00045F0040514E045F002050DE045F020050AE062690B9801219047682802D045F05D
:2046C000080505E045F4006562690B9801219047C4E9015765283DD019DC58287AD00CDC9D
:2046E000452837D004DC252826D041289ED131E046282FD0472899D12CE05B2877D0612895
:2047000028D063287CD0642823D15AE0F6E06F2848D008DC66281DD067281BD0692821D030
:204720006E2816D127E0702845D0732868D0752847D078280DD14DE0A1690D98884725284B
:2047400005463FF469AFE1690D9888476D1C3FF46AAFD8E00D9923466A466FF00100AFF3B7
:204760000080C5E045F0400023464FF000026060A80736D43EE0E8077FF447AF2068011D60
:2047800021600068290501D506701BE7290701D5068017E7A90703D5F117C0E9006111E798
:2047A00006600FE745F0400023464FF008026060A80716D41EE040F60E0125EA010060600A
:2047C00016E045F0400023464FF00A026060A80707D40FE045F040006060A80708D5234657
:2047E00010220D996FF00100AFF3008080E007E0102223460D996FF00100FEF73DFE77E0F0
:204800004FF0000963284F46C8464B46CB4602D05B2806D038E0E80601D40120A060012731
:2048200032E06269D4F80CB00B98012190475E2807D14FF0010949466269D4F80CB00B984B
:204840009047216939B900210A4603AB43F82120491C0829FADBD8B3216949B308F10108EC
:2048600062690B98012190475D28F4D1B9F1000F09D0002003A951F82020D24341F8202012
:20488000401C0828F7DB03AB2069002820794FEA40701ED05B462246CDF80080CDE901974F
:2048A0000D9900286FF0010020DAAFF300801FE0C11703AA00EBD1614B1121F01F0102EB93
:2048C0008302411A13680120884003431360C7E719E00D99224600286FF00100009702DA2B
:2048E000AFF3008004E0AFF3008001E0AFF3008000280ADA401C06D10C9820B14FF0FF306B
:204900000FB0BDE8F08F5046FAE7E90701D10AF1010A064400200C9054E60000CCCCCC0CC5
:2049200070B516460C46054600F040F8036893F80101012806D0FF2C0FD8185D68B1012079
:204940002C7070BDD3F807013246214603F2071303442846BDE8704018474FF0FF3070BDC9
:20496000754600F0E3F8AE4605006946534620F00700854618B020B5FEF7BCFCBDE820403F
:204980004FF000064FF000074FF000084FF0000B21F00701AC46ACE8C009ACE8C009ACE8A2
:2049A000C009ACE8C0098D467047000010B500F005F8001D10BD00BF294200000048704782
:2049C000740200202DE9F0411F46044603260168072A01F4006004DB08B116A505E016A540
:2049E00003E008B115A500E015A521F010002060A069C01EA0610FB1401EA0612046FEF7C4
:204A000078FE4FB1D4E9012138469047206A401C2062C01C206206E0206AFAE7D4E90121F6
:204A200015F8010B9047761EF8D22046FEF777FEBDE8F0814E414E006E616E00494E46004B
:204A4000696E66002DE9F047814616468AB0334878440DC88DE80D0030487844801C03AC62
:204A60000DC884E80D0041F69B300844372190FBF1F290FBF1F5A5F1800501FB12041B3CDF
:204A800002D56442012000E00020DFF890A080460027FA44AAF1BE0A0DE0E00709D03246BE
:204AA000684607EB47010AEB810100F00FFB8DE8070064107F1C002CEFD1184F7F44AC3F11
:204AC00018E0E80714D007EB04100DF1180A90E80E008AE80E00C068F04201D1981908906A
:204AE000324606A903A800F0F1FA03AB83E807006D10641C002DE4D132466946B8F1000F2B
:204B000003A802D000F0CEFA01E000F0DFFAC9E90001C9F808200AB0BDE8F087E44300001D
:204B20000446AFF300802046FEF7CFFB00487047540200204FF0013C50F8042B51F8043BF4
:204B40009A4221D1A2EB0C03934313EACC1317D150F8042B51F8043B9A4215D1A2EB0C03F4
:204B6000934313EACC130BD150F8042B51F8043B9A4209D1A2EB0C03934313EACC13DBD0F9
:204B80004FF00000704700BFD01A01BAB1FA81F101F0180122FA01F0CB40C1F12001DBB21C
:204BA000C0B2C01A2CFA01F3D11A914311EAC311E6D1704701491820ABBEFEE7260002009B
:204BC00070475FEA400C08BF91F0000F4FEA8C234FEAC12243EA51514FEA1C5018BF00F5EE
:204BE000F0404FEA300018BF41F000415FEA6C5C00F02980BCF1FF3F08BF40F080407047D0
:204C0000130C06BF12044FF0100C4FF0000C130E04BF12020CF1080C130F04BF12010CF1F6
:204C2000040C930F04BF92000CF1020CD30F04BF52000CF1010C11464FF00002A0F11F0019
:204C4000A0EB0C00704711F0004F08BF704731F000413FF4D5AF0B0C06BF09044FF0100CDB
:204C60004FF0000C0B0E04BF09020CF1080C0B0F04BF09010CF1040C8B0F04BF89000CF11A
:204C8000020CCB0F04BF49000CF1010CCCF12003A0EB0C0022FA03F302FA0CF241EA030164
:204CA00000F10100704720F07F4C80EA030023F07F47ACEB070303F57C5300F0004003F19E
:204CC000FF032DE980494FEA154B09B44FEA144325EA0B4E24EA03480FF2042606EB1327F6
:204CE00049083E785FEA320203FB0667C7F5000707FB06F64FEA54374FEAD64606F10206EC
:204D000007FB066CCCF1005C4FEA1C472CEA074C07FB06F40CFB06F504EB15464FEA9616D4
:204D200034BF00204FF000404FEAD13706FB07FC4FEA1C4C0CFB0BF7D21B03FB0CF761EBB8
:204D400007010CFB0EF7B0EB074072EB17420CFB08F734BFA2EB0742B2EB074261EB17414E
:204D60004FEA0C444FEA910706FB07FC4FEA1C4C0CFB0BF7B0EBC74072EB573203FB0CF7A2
:204D800034BFA2EBC742B2EBC74261EB57310CFB0EF7B0EBC70072EB57720CFB08F734BF83
:204DA000A2EBC702B2EBC70261EB5771039F4FEA816141EA921104EBCC044FEAD1374FEA5F
:204DC000826206FB07FC42EA90124FEA80604FEA1C4C0CFB0BF7D21B03FB0CF761EB070118
:204DE0000CFB0EF7B0EB074072EB17420CFB08F734BFA2EB0742B2EB074261EB17414FEA7D
:204E00008C554FEA910704EB9C2406FB07FC4FEA1C4C0CFB0BF7B0EBC74072EB573203FBFD
:204E20000CF734BFA2EBC742B2EBC74261EB57310CFB0EF7B0EBC70072EB57720CFB08F7D2
:204E400034BFA2EBC702B2EBC70261EB577115EB4C254FEA816141EA92114FEA82624FEADF
:204E6000D13742EA901206FB07FC44F100044FEA80604FEA1C4C0CFB0BF7D21B03FB0CF76E
:204E800061EB07010CFB0EF7B0EB074072EB17420CFB08F734BFA2EB0742B2EB074261EB19
:204EA000174115EB1C154FEA813141EA92414FEA823242EA90424FEA80304FEA0C7644F1BC
:204EC000000448EA03434EEA0B484FF0000EB2EB080C71EB030724BF624639464EEB0E0E08
:204EE0004FF0000B0018524149414BEB0B0BB2EB080C71EB03077BF1000B24BF624639464F
:204F00004EEB0E0E4FF0000B0018524149414BEB0B0BB2EB080C71EB03077BF1000B24BF00
:204F2000624639464EEB0E0E51EA020718BF46F0010616EB0E7655F1000254F1000103D5B2
:204F4000BDE88901BDE80088BDE88901BDE80048B619524141EB0101A3F1010370478080FA
:204F60007F7E7D7C7B7A7978777676757473727171706F6E6E6D6C6C6B6A6A6968686766FD
:204F800066656464636362616160605F5F5E5E5D5D5C5C5B5B5A5A5959585857575656556D
:204FA00055555454535352525251515050504F4F4F4E4E4D4D4D4C4C4C4B4B4B4A4A4A4915
:204FC000494948484847474747464646454545444444444343434342424242414141002B98
:204FE00026D4770021D01CB54FEA370703B44FF010004FF010014FF000000FBCBDE81040B2
:205000000BF1010BBBF1010F08BF5FEA170722BF12F1010211F101014FF0004143F10003FC
:2050200000F0004043EA00007047F9D35708DAE746EA064613F1400F4FEA16461FDD13F10C
:20504000200FDFBF16430A46002120335B42C8D0C3F1200746EA064602FA07F74FEA16464B
:2050600046EA0706C3F1200722FA03F201FA07F721FA03F14FF0000342EA0702B1E746EAC0
:20508000020646EA06464FEA164646EA0106BCBF46EA0646360C4FF000034FF000024FF0C5
:2050A00000019EE72DE9C048934630B491E8380007C831EA400C48BF34EA430C03D5FFF766
:2050C000F2FDFFF78CFFF0BCBDE800882DE9C048934630B491E8380007C810F0804F08BF96
:2050E00013F0804F03D100F005F8FFF778FFF0BCBDE8008820F07F4780EA030023F07F4CB6
:2051000007EB0C03A3F57C5300F00040A3F1FE0392F0000F00F0B38095F0000F00F0778033
:205120002DE901494FEA11404FEA144621EA004800FB06FC24EA064708FB06F607FB08F846
:2051400000FB07F718EB06484CEB164C4FEA124B18EB07484FEA15464CEB174022EA0B4EFD
:205160000BFB06FC25EA06470EFB06F607FB0EFE0BFB07F71EEB064E4CEB164C4FF0000679
:205180001EEB074E4CEB174B18EB0B0840F1000018EB0E0B58EB000840F100008F1A4FF051
:2051A00000013CBFC943661B14BFB5EB040C00213CBFC943F61B4FEA17444EEA8E0E27EA31
:2051C00004454FEA1C4704FB07622CEA074C05FB07F70CFB05F604FB0CFC16EB074642EB97
:2051E000174216EB0C4642EB1C421BEB060658EB0202414146EA9E0601D5BDE80189B619F5
:20520000524141EB0101A3F10103BDE801894FEA14454FEA114724EA054621EA074C05FB2C
:2052200007F406FB07F70CFB06F105FB0CFC11EB074144EB17444FEA124711EB0C4144EB96
:205240001C4422EA074C05FB07F206FB07F70CFB06F605FB0CFC16EB074642EB174216EBB7
:205260000C4642EB1C456A1854F1000148BF7047B619524141EB0101A3F10103704795F064
:20528000000F37D04FEA11424FEA144721EA024624EA074C02FB07F106FB07F70CFB06F42F
:2052A00002FB0CFC14EB074441EB17414FEA154714EB0C4441EB1C4125EA074C02FB07F553
:2052C00006FB07F70CFB06F602FB0CFC16EB074645EB174516EB0C4645EB1C42121951F19F
:2052E000000148BF7047B619524141EB0101A3F1010370474FEA14454FEA114724EA054694
:2053000021EA074C05FB07F106FB07F70CFB06F24FF0000605FB0CFC12EB074241EB174122
:2053200012EB0C4251EB1C4148BF7047921841EB0101A3F10103704710B500F010F8C0F334
:20534000401010BD10B50E2000F016F804460F2000F012F804F00F0140EA012010BD0B2085
:2053600000F00AB810B54FF0FF34FFF7E5FF08B1002010BD204610BD1FB54FF47A7301226A
:2053800003A98DE80E00134602466C21034801F0AFF89DF80C0004B010BD00007400002017
:2053A000FEE70000014800F0A7BA00004C000020014800F0FBBC00005001002030B590F834
:2053C000444004F01C050124AC40056C6C60046863608368102B036803D099600068C260D0
:2053E00030BD9A600068C16030BD704772B6FEE7144A117F1448012901D003290FD10368D0
:2054000023F400730360036843F400630360036823F400630360036843F40073036002294C
:2054200001D003290BD1016841F480510160016821F480510160016841F480610160002013
:20544000107770470C00002000200240C107054803D0416941F004014161416941F4803186
:20546000416170470020024008494A69C0B222F47E7242EAC0004861486940F002004861D4
:20548000486940F4803048617047000000200240054910B54C6944F001044C610260BFF3F3
:2054A0006F8F436010BD000000200240094A10B55469402344F480245461EFF3108272B6B7
:2054C00010C910C05B1E13F0FF03F9D182F3108810BD00000020024070B5054600F050FFF0
:2054E0000646134C08E0681C06D000F049FF801BA84201D3032070BD2069C003F3D4206942
:205500000C4908400CD00C494A6802434A60810F01D0A169A161810000D02061012070BD8F
:205520002069C00701D001202061002070BD000000200240FAC302000C00002001884088BD
:205540004AF25A52514040BA4840704710B50446012020800020A070E0702046FFF7EEFF00
:20556000A08010BD70B5114801684068CA4372EA000215D08BB20C0C0D4A44EA0044090E2A
:205580001380947041EA0021D17090801446B3F5006F05D21046FFF7D1FFA188884202D0AE
:2055A0000348FFF7D3FF024870BD000000F803084400002070B586B00446FFF7BFFFA08081
:2055C000A17822880B0CE47842EA0141220A1A43002541EA046440EA020600F0C7FD7F2061
:2055E000029001200390009504A9684600F0F6FC044922463346002000F066FD00F05AFDAB
:2056000006B070BD00F8030890F82020012A07D0022A05D0416A41F48021416201207047DD
:20562000006842690A43426100207047F0B590F820500468A468012D05D0022D03D0416ACB
:2056400041F480214DE014F0406F01D1E50045D5C4F301640125A5401D608D684FF4C073B4
:205660009DB1CE6835434E6845EAC605066803EB0417F5514FF4C275076805EB04150E6958
:205680007E51097D012905D009E00E88CD6845EA4655EBE701684E5946F480764E511179FD
:2056A000D2F805504FF4C67641EA0521056806EB0416A9511178D2F801204FF4C47541EA6E
:2056C0000221026805EB04155151006803EB0411425842F0010242500020F0BD416A41F419
:2056E000001141620120F0BD10B590F82020012A07D0022A05D0416A41F480214162012053
:2057000010BD0068D0F8002242F00102C0F800220A7D02F01F0301229A40D0F81C329343D7
:20572000C0F81C32CB69B3B9D0F80C329343C0F80C328C894B6864F31F434C6900EBC40408
:20574000C4F840320C890B6864F31F434C6900EBC404C4F84432CB69012B16D1D0F80C3273
:205760001343C0F80C320C884B6864F31F434C6900EBC404C4F840320C89CB6864F31F43C6
:205780004C6900EBC404C4F844328B69002BD0F804320FD053EA0203C0F804320B69002BA4
:2057A000D0F8143208D01343C0F81432096A012904D008E09343EFE79343F5E7D0F81C1202
:2057C0001143C0F81C12D0F8001221F00101C0F80012002010BD704770B590F82040012CFA
:2057E00005D0022C03D0416A41F4802128E0046809B32469A40720D04FF4D874056804EB0F
:2058000001142D5915F00405956005682D591AD0ED08556005682C5904F00204D4604FF400
:20582000DA74056804EB01142E5906F00F06082E0CD308250DE0E468DCE7416A41F40011E8
:205840004162012070BD6D0D1560E3E72D5905F00F05156105682D59C5F30725956105685F
:205860002C59240C54614FF4DC72046802EB0112A4581C700468A458240A5C700468A4586F
:20588000240C9C700468A258120EDA704FF4DE72046802EB0112A4581C710468A458240ADE
:2058A0005C710468A458240C9C710468A258120EDA71006829B1016941F020010161002025
:2058C00070BDC16841F02001C160F8E70246002092F82010012901D002290CD111688A6890
:2058E000520100D501208A68120100D5401C8968C90000D5401C70472DE9F05F054600686F
:2059000000244669D0F804908768D0F80CB0D0F810A0D0F81880F10748D0F90714D00121F7
:205920008160B80703D5284600F0EBF90CE0780702D54FF4006407E0380702D54FF48054B0
:2059400002E0284600F0DCF9F80516D529684FF480708860B80503D5284600F0D4F90CE0F2
:20596000780502D544F4005407E0380502D544F4804402E0284600F0C5F9F80316D52968DB
:205980004FF480308860B80303D5284600F0BDF90CE0780302D544F4004407E0380302D5D2
:2059A00044F4803402E0284600F0AEF9300707D55FEACB6004D52968102044F40074C8601F
:2059C00070074FF0080707D55FEA0B7004D52868C760284600F058F9B00706D52868C068D9
:2059E000800702D0284600F051F9700607D55FEACA6004D52968102044F480640861B0060C
:205A000007D55FEA0A7004D528680761284600F047F9F00606D528680069800702D02846E7
:205A200000F03FF9B00308D55FEAC96005D5296810204860284600F035F9F00307D55FEA55
:205A4000097004D528684760284600F05FF9300446D55FEA497040D5F00504D55FEAC87052
:205A600001D044F00104B00504D55FEA887001D544F00204700504D55FEA487001D544F0E4
:205A80000404300529D518F0700F26D008F07000402815D006DC102809D020280AD030282C
:205AA00016D10AE050280ED0602811D10EE044F008040DE044F010040AE044F0200407E0C9
:205AC00044F0400404E044F0800401E044F480742868816921F0700181612968042048606A
:205AE000002C05D0686A204368622846FFF773FEBDE8F09F70B5040003D094F8200010B134
:205B000004E0012070BD204600F082F82068016841F00101016000F033FC0546052604E085
:205B200000F02EFC401B0A2811D820684068C007F6D02068016821F00201016000F020FCA6
:205B400005460BE000F01CFC401B0A2806D9606A40F40030606284F82060D2E720684068C6
:205B60008007EFD4207E0128206801683DD021F080010160607E01282068016838D021F012
:205B800040010160A07E01282068016833D021F020010160E07E0128206801682ED041F0EE
:205BA00010010160207F01282068016829D021F008010160607F01282068016824D021F048
:205BC00004010160D4E902010843D4E90412114308436168491E08432168C86100206062D3
:205BE000012084F82000002070BD41F08001C0E741F04001C5E741F02001CAE721F01001FF
:205C0000CFE741F00801D4E741F00401D9E7000010B586B0044614216846FDF740FD17492A
:205C20002068884227D11648816D41F000718165816D01F000710591C16C41F00201C164DA
:205C4000C06C694600F0020005904FF4407000900220019000200290032003900920049087
:205C6000084800F097FA00221146142000F090FD142000F07FFD06B010BD00000064004062
:205C8000001002400004004870470000024B034A0021FFF7A1BD0000340000201802002012
:205CA000704770477047000070B5044690F82000012804D0606A40F40020606218E00220B1
:205CC00084F820002068016821F00101016000F057FB05460EE000BF00F052FB401B0A28BF
:205CE00008D9606A40F400306062052084F82000012070BD20684068C007EDD1606270BD20
:205D0000704770477047704770477047704710B540B190F825100022022905D00421C163A4
:205D200080F82420012010BD01680B6823F001030B6001680B6823F00E030B6090F8441014
:205D4000046C01F01C03012101FA03F3636080F8251080F82420002010BD10B590F8251015
:205D60000024022903D00421C16301241AE001680A6822F001020A6001680A6822F00E0242
:205D80000A6090F84410036C01F01C02012101FA02F25A6080F82510002180F82410816B0E
:205DA00001B18847204610BDC06B7047F0B4016C0D6801680C6890F8442002F01C060422C4
:205DC00002FA06F32B4211D063070FD50B689B0603D40B6823F004030B6090F8441001F082
:205DE0001C018A40016C4A60016B26E0022202FA06F72F424FF0000C4FF0010321D0A70778
:205E00001FD50C68A40605D40C6824F00A040C6080F82530184B0168994290F8441001F054
:205E20001C0102FA01F202D914490A6002E0124980394A6080F824C0C16A00291AD0F0BCCE
:205E400008470822B2402A4214D0220712D50A6822F00E020A6090F84410026C01F01C0121
:205E600003FA01F15160C36380F8253080F824C0416BE2E7F0BC704780000240040402404F
:205E800010B568B12C4C026814232C49A24209D22B4C1444B4FBF3F39B00C0E910130BE021
:205EA000012010BD244C64421444B4FBF3F39B004364214B083B0364022380F8253013682C
:205EC00047F6F074A3431360D0E902231A43D0E9043423431A4383691A43C3691A43036A9A
:205EE0001A4303681C6822431A608268B2F5804F19D0036C0F228B4202D151F8A83F02E0DC
:205F00000D49A0310B6890F8444004F01C04A24093430B6090F84430426803F01C039A4012
:205F20000B681A430A600021C163012280F8252080F82410084610BD0804024000000240AB
:205F4000F8FFFDBF70B5044690F82400002501280ED0012084F8240094F825600020012E26
:205F600008D08021E16384F824000125284670BD022070BD022684F82560E0632068066852
:205F800026F0010606602046FFF718FA206B00282068016802D041F00E0106E021F004015E
:205FA00001602068016841F00A0101602068016841F001010160D9E770B5044600F0E0F975
:205FC0000546601C02D004480078044400F0D8F9401BA042FAD370BD000000202DE9F05F9F
:205FE000054632488946017801290CD00126804606704CF2503B5846FFF76EFA07004FF020
:20600000000A03D04EE00220BDE8F09F51464046C8F804A0264C226892050AD52168490555
:2060200005D5216821F480612160032109E0067708E02268520504D5216821F4806121605A
:20604000022101772868012807D04FF0FF31C9F8001040F2FA3BAE681DE06868FFF7F6F9A6
:206060005846FFF739FA0746606920F00400606116E030466968FFF7F7F94CF25030FFF797
:206080002BFA0700606920EA0B00606102D0C9F8006005E0761CD5E902010844B042E8D80C
:2060A000FFF7A6F988F800A03846ADE70C000020002002400348416941F000414161002062
:2060C00070470000002002402DE9FF5F254C0646904620789A4601280BD0012020704CF235
:2060E000503B5846FFF7F8F907004FF0000904D02AE0022004B0BDE8F09F4846C4F804907B
:20610000194D2968490504D5286820F4806028600220207726B1012E09D0022E07D00CE0CA
:20612000424653460198FFF7B3F9012612E041460198FFF7BBF9022E0AD05846FFF7CCF9BD
:206140004FEA0007FFF754F984F800903846D1E74FF480265846FFF7BFF907466869B04334
:206160006861EFE70C00002000200240064900204A69002A07DA054A8A60054A8A604969A1
:20618000002900DA012070470020024023016745AB89EFCD2DE9F04FDFF8AC91002303254E
:2061A000A9F1040B85B04FF0010C0F2709F1040AABF1040EBFE000BF0CFA03F6324075D0B5
:2061C0000C7904F00304012C01D0022C1BD1846800945C0005FA04F80494009C24EA080402
:2061E0000094D1F80C80049C08FA04F8009C48EA0408C0F808804468B4430E79C6F3001605
:206200009E40264346600C79E443A4070AD0C4684FEA430805FA08F6B4438E6806FA08F6C8
:206220002643C6600C7904F00304022C10D1DC0800EB84040294246A5E074FEAD66807FAE8
:2062400008F6B4430E6906FA08F62643029C266204684FEA430805FA08F6B4430E7906F0E4
:20626000030606FA08F6264306604C6814F4403F60D0364C266E46F001062666246E23F059
:20628000030604F001040094314C34440294A4689E074FEA167807FA08F6B443B0F1904FEF
:2062A00005D02C4EB04204D1012612E042E000260FE0294EB04201D102260AE0274EB042C4
:2062C00001D1032605E0264EB04201D1042600E0072606FA08F62643029CA660D9F8006033
:2062E0004C46D1F8048096435FEAC82800D516432660DAF800405646D1F8048094435FEADE
:20630000882800D514433460DBF800405E46D1F8048094435FEA883800D514433460DEF893
:2063200000407646D1F8048094435FEAC83800D5144334605B1C0A6832FA03F47FF43CAFCA
:2063400005B0BDE8F08F00000804014000100240000001400004004800080048000C004894
:2063600000100048426921EA02030A4043EA0241816170470AB181617047816270470000C9
:2063800001488068704700000000002090F84120202A24D190F84020012A20D0012280F82F
:2063A0004020242280F841200268136823F0010313600268136823F48053136002681368C8
:2063C0000B43136001680A6842F001020A60202180F84110002180F8401008467047022068
:2063E000704790F84120202A22D190F84020012A1ED0012280F84020242280F8412002683B
:20640000136823F0010313600268136823F4706343EA0121116001680A6842F001020A606E
:20642000202180F84110002180F84010084670470220704770B5040004D094F8410000259C
:2064400010B106E0012070BD84F84050204600F001F9242084F841002068016821F00101E6
:2064600001606068216820F0706008612068816821F400418160E0680128A06830D040F4CC
:20648000044021688860E0680228206841682AD021F40061416020684168144A114341600F
:2064A0002068C16821F40041C160D4E904010843A16940EA01202168C860D4E90701084391
:2064C000216808602068016841F0010101606564202084F84100256384F84250002070BD9D
:2064E00040F40040CDE741F40061D3E7008000022DE9FF4F83B00446DDE9108790F841009B
:20650000DDF848A09B46202876D15FEA080015D0A7B194F8400001286ED04FF0010984F8C8
:206520004090FFF72DFF0646012200901923D103204601F08FFA002872D103E04FF4007079
:2065400060646DE0222084F84100402084F8420000256564C4F8248067856563CDE900A6AF
:20656000DDE904125B46204601F02AFA10B184F8405055E0618D35484FF080774FF00078C9
:20658000FF2905D9A4F828904A463B46009005E0618D2185009094F8282043462046049997
:2065A00001F040FA5346002204212046009601F051FAA8BB2068406A616A0870606A401C9A
:2065C0006062208D401E81B22185608D401E6085608DE0B1D9B9534600228021204600967D
:2065E00001F038FAE0B9608DFF2806D9A4F828904A463B46009506E026E0608D20850095DF
:2066000094F8282043462046049901F00BFA608D0028C7D132465146204601F058FA18B1F6
:20662000012007B0BDE8F08F21682020C86121684A68074B1A404A6084F8410084F8425010
:2066400084F840500020ECE70220EAE70024008000E800FE30B59DB00446142117A8FDF75A
:206660001EF85C216846FDF71AF817492068884228D18020002500900D95684600F0F6F8A5
:2066800008B1FEF7B3FE114CE06C40F00200E064E06C17A900F002001C904FF4C0401790E8
:2066A0001220CDE9180503201A9004201B900848FFF770FDA06D40F48000A065A06D00F4BF
:2066C00080001C901DB030BD00580040001002400004004802488168027811448160704704
:2066E0000000002010B50024032000F071F80F2000F008F808B1012401E000F025F82046C4
:2067000010BD000070B50E4E05460024307898B14FF47A71B1FBF0F00A490968B1FBF0F0C1
:2067200000F0C6FD40B9102D06D200222946501E00F02EF8756000E00124204670BD000016
:20674000000000202C000020094808B5016E41F001010166016E01F001010091816D41F0A4
:2067600080518165806D00F08050009008BD000000100240002809DB00F01F0201219140FE
:206780004009800000F1E020C0F8001170470000F0B40E4B1B680C46C3F30223C3F1070552
:2067A000042D00D90425191D072901D2002300E0DB1E012606FA05F1491E214099409E40D5
:2067C000761E16403143F0BC01F0DDBF0CED00E0064900F0070208684FF6FF03184040EAC8
:2067E0000220034A10430860704700000CED00E00000FA051649B0F5007F0868C0F34120D9
:2068000009D0022805D0086820F4C06040F480600860002070470128FBD0086820F4C06011
:2068200040F4007008600B483222006850430A4AB0FBF2F0401C00E0401E4A69520501D54F
:206840000028F9D148694005E3D5032070470000007000402C00002040420F00024800687F
:2068600000F4C06070470000007000402DE9F84F044600270088A84D3E46000515D5606C13
:2068800060B1B0F5000F04D0B0F5400F2BD001270AE0E86840F48030E86024E00021201D80
:2068A00001F03AFA07001ED03E46206880033AD5A86D4FF00008C00009D4A86D40F0805012
:2068C000A865A86D4FF0010800F080500090DFF84CA2DAF8001041F48071CAF80010FFF769
:2068E0004FFD814610E0D5F88800616C20F440000843C5F88800D8E7FFF742FDA0EB090007
:20690000022801D9032705E0DAF80000C005F3D5002F7DD04FEA0706B8F1000F03D0A86DA3
:2069200020F08050A8652078C00707D0D5F88800216A20F003000843C5F888002078800792
:2069400007D5D5F88800616A20F00C000843C5F888002078400707D5D5F88800A16A20F064
:2069600030000843C5F888002078800607D5D5F88800E16A20F440600843C5F888002088D1
:20698000800507D5D5F88800E16B20F440200843C5F888002088400507D5D5F88800216C46
:2069A00020F440100843C5F888002078400607D5D5F88800216B20F440500843C5F8880014
:2069C0002078000607D5D5F88800616B20F440400843C5F888002088C00507D5D5F888005A
:2069E000A16B20F440300843C5F8880020684FF0006700034FF0806850D5D5F88800A16C98
:206A000020F040600843C5F88800A06CB84200E005E03BD1E86840F48010E8603EE0D5F818
:206A2000900010F4407014D0A16D814211D0D5F89000D5F8901020F4407041F48031C5F84B
:206A40009010D5F8901021F48031C5F89010C5F89000C00711D0FFF793FC074641F288394B
:206A600007E000BFFFF78CFCC11B494501D9032652E7D5F890008007F4D5D5F89000A16D34
:206A800020F440700843C5F8900045E7404505D10121201D01F040F900B1064620684003C2
:206AA00017D5D5F88800E16C20F040600843C5F88800E06CB84204D1E86840F48010E86091
:206AC00007E0404505D10121201D01F025F900B106462088400411D5D5F88800216D20F044
:206AE00040500843C5F88800206DB0F1805F05D10221201D01F010F900B106462088000490
:206B000006D555F8880F616D20F08040084328603046BDE8F88F00000010024000700040A1
:206B20002DE9F0470F4605006BD0494E306800F00700B84209D2306820F0070038433060BE
:206B4000306800F00700B8425BD12878414C80070AD5A868A16801F0F001884204D9A16842
:206B600021F0F0010143A1602878C0072CD06868032811D0022812D0216898B1490500293A
:206B80003FDAA16821F003010143A160FFF7F8FB804641F2883910E021688901EFE7216874
:206BA0008903ECE78907EAE7FFF7EAFBA0EB0801494502D90320BDE8F087A068696800F035
:206BC0000C00B0EB810FEFD1287880070AD5A868A16801F0F001884204D2A16821F0F00112
:206BE0000143A160306800F00700B8420BD9306820F0070038433060306800F00700B842A0
:206C000001D00120D7E72878400705D5A068E96820F4E0600843A0602878000706D5A06881
:206C2000296920F4605040EAC100A06000F03EF8A168094AC1F30311515C01F01F01C84003
:206C40000649086006480068BDE8F047FFF75ABD00200240001002400C8D00082C0000203D
:206C6000040000200548064900688968054AC1F30221515C01F01F01C84070472C0000200C
:206C8000001002404C8D00080548064900688968054AC1F3C221515C01F01F01C840704769
:206CA0002C000020001002404C8D000870B52449002318468A68CC6812F00C0204F003060F
:206CC000204C214D09D00C2A05D0042A32D0082A00D1284670BD012E10D10B681B0704D4AB
:206CE000D1F89430C3F3032302E00B68C3F30313164E56F82330DAB10C2AEBD1C86800F068
:206D00000300022818D0032818D01846CA68CB68C2F30212C3F306234343521CB3FBF2F25A
:206D2000C868C0F34160401C4000B2FBF0F070BD184670BD204670BD2046E7E72846E5E7ED
:206D4000001002400024F40000366E011C8D00082DE9F84304006FD0FA4DA86800F00C0686
:206D6000E86800F003072078C00664D576B10C2E01D1012F0AD0A069002828687AD040F0BA
:206D800001002860FFF7FCFA80465DE02868800702D5A0690028DED0216A2868000703D5B4
:206DA000286800F0F00004E0D5F89400F02202EA1010814216D9084601F044F800283BD19F
:206DC000286840F0080028602868216A20F0F000084328606868E16920F47F4040EA01203D
:206DE000686016E0286840F0080028602868216A20F0F000084328606868E16920F47F40AA
:206E000040EA0120686026B9206A01F01BF80028D5D1FFF74BFFA968CB4AC1F30311515C49
:206E200001F01F01C840C9490860C9480068FFF769FC00287ED12EE0CAE000BFFFF7A0FA6D
:206E4000A0EB0800022876D828688007F6D5286840F0080028602868216A20F0F00008438F
:206E600028606868E16920F47F4040EA0120686011E0FFE720F001002860FFF781FA8046E3
:206E800006E000BFFFF77CFAA0EB08000228DAD828688007F6D42078C00740D0082E18D004
:206EA0000C2E01D1032F14D06068B0F5803F17D0B0F5A02F286817D020F4803028602868D6
:206EC00020F4802028606068E0B1FFF759FA804614E02868800322D56068002878D01EE0DA
:206EE000286840F48030EDE740F480202860F7E7FFF746FAA0EB08006428A4D8286880032C
:206F0000F6D50CE0FFF73CFA804605E0FFF738FAA0EB0800642896D828688003F6D42078B9
:206F200080073BD5042E11D00C2E01D1022F0DD0E06801E0AAE1FFE0002828681ED040F420
:206F400080702860FFF71CFA07460CE0286840050CD5E0680028C1D008E000BFFFF710FA16
:206F6000C01B022893D828684005F7D56868217C20F0F85040EA016068600FE020F48070F5
:206F80002860FFF7FDF9074605E000BFFFF7F8F9C01B0228B1D828684005F7D420780007D8
:206FA00029D560690028D5F8940012D040F00100C5F89400FFF7E4F9074604E0FFF7E0F94A
:206FC000C01B022899D8D5F894008007F6D512E02BE120F00100C5F89400FFF7D1F907461B
:206FE00005E000BFFFF7CCF9C01B022885D8D5F894008007F6D42078400766D5A86D0027C8
:20700000C00008D4A86D40F08050A865A86D012700F0805000904F480168C90512D4016808
:20702000814641F480710160FFF7AAF9804605E0FFF7A6F9A0EB080002287DD8D9F8000046
:20704000C005F5D5A068012816D00528D5F8900017D020F00100C5F89000D5F8900020F04E
:20706000040000BFC5F89000A06841F28839C0B1FFF786F980460FE0D5F8900040F00100DB
:20708000F0E740F00400C5F89000F5E7FFF778F9A0EB080149454FD8D5F890008007F5D55E
:2070A0000EE0FFF76DF9804606E000BFFFF768F9A0EB080149453FD8D5F890008007F5D4DE
:2070C0001FB1A86D20F08050A8652078800628D5606A0028D5F8980012D040F00100C5F89C
:2070E0009800FFF74DF9074605E000BFFFF748F9C01B022820D8D5F898008007F6D510E0F0
:2071000020F00100C5F89800FFF73AF9074604E0FFF736F9C01B02280ED8D5F898008007B3
:20712000F6D4A06AF0B3022816D00C2E7DD0286820F08070286000E0A7E0FFF721F9044668
:20714000A6E00000001002400C8D00082C0000200400002000700040E868E26A00F0030106
:20716000914228D1216B00F0700209011039914221D1626B00F4FE41B1EB022F1BD194F8F8
:20718000382000F07841B1EBC26F14D1A18F00F4C00249084905A1F5001191420BD194F8D5
:2071A000401000E06AE04908490600F0C060A1F1007181424BD00C2E73D02868400170D432
:2071C000286820F080702860FFF7DAF8064604E0FFF7D6F8801B022857D828688001F7D40B
:2071E000F4E90B016FF00F0202EB01110843218A5204490802EB4151A26841EA0221084378
:20720000217D4FF07E42490802EB41610843217B40EAC160E968244A11400843E86028688C
:2072200040F080702860E86800E03AE040F08070E860FFF7A5F8044605E000BFFFF7A0F8E5
:20724000001B022821D828688001F7D527E02868800124D4286840F080702860E86840F04B
:207260008070E860FFF78CF8044604E0FFF788F8001B022809D828688001F7D50FE000BF07
:20728000FFF77EF8001B022802D90320BDE8F88328688001F4D4E86804490840E8600020F9
:2072A000F4E70120F2E700008C809D01FCFFEEFE10B5401EB0F1807F01D3012010BD4FF0A4
:2072C000E02460610F21601701F05DFA0020A06107202061002010BD7047704770B5044667
:2072E000C06FD4F88060216889684FF01005090618D5212816D12068083050E8001F21F091
:20730000800140E80012002AF5D1206F38B1FEF7FEFC20B1206FFEF747FD202821D0204623
:2073200001F065F820688068400618D5222E16D12068083050E8001F21F0400140E8001282
:20734000002AF5D1606F38B1FEF7E1FC20B1606FFEF72AFD202804D0204601F022F800204A
:2073600070BDC4F88450032070BD000010B5044600680A49884210D12046FFF7AFFF084930
:207380000020087020210748FCF767F92046BDE810402022034900F0FFB910BD003801409B
:2073A0003C000020340200202DE9F04102680446D0691168936840F60F0528424FF000057B
:2073C0004FF0020605D187067ED58F067CD5A16E33E1DFF894C203F0010701EA0C0C57EA3B
:2073E0000C0C71D05FEAC07C0CD05FEAC15C09D54FF0010CC2F820C0D4F8842042F0010204
:20740000C4F88420820709D5DA0707D022681662D4F8842042F00402C4F8842042070AD5BB
:20742000DA0708D0236804221A62D4F8842042F00202C4F8842002070CD501F020023A43E6
:2074400008D0236808221A62D4F8842042F00802C4F8842002050BD54A0109D523684FF439
:2074600000621A62D4F8842042F02002C4F88420D4F88420002A36D0800605D5880603D5A4
:20748000A16E09B120468847D4F8840021688968490602D410F0280F27D0204600F081FFFB
:2074A0002068806840061BD52068083050E8001F21F0400140E80012002AF5D1606F78B19B
:2074C0006A498163606F00E015E0FEF746FC002809D0606F816B00E02046BDE8F041084713
:2074E0002046FFF743FFBDE8F0812046FFF73EFFC4F88450F7E7D4F860C02027BCF1010FE1
:207500007ED15FEAC06C7BD55FEAC16C78D5102010622068806840064FD5616F0A6850681E
:207520000004000C3DD0B4F85830834239D9A4F85A000868006880062BD4206850E8001FF1
:2075400021F4807140E80012002AF6D12068083050E8001F21F0010140E80012002AF5D1A6
:207560002068083050E8001F21F0400140E80012002AF5D1C4F880702566206850E8001F62
:2075800021F0100140E80012002AF6D1606FFEF7BEFB6666B4F85800B4F85A10401A81B2AE
:2075A00007E0B4F8581081429DD1106880069AD566662046FFF790FE95E7B4F85800B4F850
:2075C0005A10401A81B2B4F85A0000288BD0002989D0226852E8000F20F4907042E8000395
:2075E000002BF6D12068083050E8002F22F0010240E80023002BF5D1C4F88070256600E00A
:207600000AE0A566226852E8000F20F0100042E80003002BF6D1CBE7C60209D55B0207D5D2
:207620004FF4801010622046BDE8F041FFF755BE020606D50A0604D5E16E00297FF44CAF0E
:2076400051E74006B8D54806B6D52046026852E8001F21F0400142E80013002BF6D1C7676E
:20766000C56600F015F93EE7200100048582000810B5040002D0E06F10B107E0012010BD08
:20768000002084F87800204600F026F82420E0672068016821F001010160606A10B1204681
:2076A00000F050FC204600F0AFFE0128E7D02068416821F4904141602068816821F02A0146
:2076C00081602068016841F0010101602046BDE8104000F09BBC0000F0B59DB0064614212F
:2076E00017A8FBF7DCFF5C216846FBF7D8FF26493068884245D101240025684608950094FA
:20770000FFF7B4F808B1FDF771FE2048016E41F480410166016E01F480411C91C16C41F047
:207720000101C164C06C022700F001001C904FF4C060CDE917070320CDE9194007201B90F5
:2077400017A94FF09040FEF725FD124C10482060C4E901758020C4E903506561A561E56138
:2077600020462562FEF78CFB08B1FDF73FFE7467002211462520A662FFF70AF82520FEF7E3
:20778000F9FF1DB0F0BD00000038014000100240580002405001002030B4D0F88030202BFA
:2077A00002D0022030BC7047A9B1A2B1002303660A4C0368A3420BD05B681B0208D504684F
:2077C00054E8003F43F0806344E80035002DF6D130BC00F019BF0120E4E700000080004063
:2077E000704770472DE9F84F0446C06F984615460E46202802D00220BDE8F88F86B37DB3E7
:207800000020C4F884004FF02109C4F87C90FEF7B7FDA4F850508246A4F85250A068B0F53F
:20782000805F01D1206910B13546002600E000255FF02007B4F8520053464FF00002CDF894
:207840000080D0B18021204600F02EFFD0B94DB115F8010B21688862E16F39EA010006D0A6
:207860000120C9E736F8020BC0F30800F2E7B4F85200401EA4F85200DCE74021204600F0A4
:2078800013FF10B1E7670320B6E7E7670020B3E77047FEE701688A69D243920701D4002262
:2078A0008A6200688169C943C90703D0816941F001018161704700002DE9F0470446006826
:2078C00088460026816935461746C9064FF020093FD51021C1612FE0B8F1FF3F2CD0FEF76D
:2078E0004FFDC11B414502D8B8F1000F24D12068416894F8422001F480418369DB431B0455
:2079000015D4B1F5804F12D0202A10D0416841F480414160FEF734FD074608E0FEF730FD40
:20792000C01B192803D945F02005012604E020688069C0438006F1D420688069C0F34010B7
:207940003043C9D016B92168C1F81C9045F00405012621688869C20505D54FF4807245F074
:207960000105CA610126410509D522684FF4806145F00805D1610126800502D40AE0800578
:2079800007D521684FF4007045F00205C861012600E086B12046FFF77DFF54F8241B486819
:2079A000064A10404860206A2843206284F81D900020A07720773046BDE8F08700E800FE99
:2079C0002DE9F84304461646DDE9089714489846DAB200900023204600F024F83A46494651
:2079E000204600F09FF8B8B9F5B2B8F1010F08D02168300A88623A464946204600F092F855
:207A000050B9206885624B46002240212046009700F020F8002800D00120BDE8F88300009C
:207A20000020008010B5C1F3090141EA02410268029C19432143506821F000414FF48063BD
:207A400003EA5453024C234398430843506010BDFF63FF032DE9F0411D4617460E46044632
:207A6000DDF8188027E0424629462046FFF724FF10B10120BDE8F081681C1CD0FEF780FC43
:207A8000A0EB0800A84200D8ADB92068806936EA00000ED00020B8420DD154F8440F40F0F5
:207AA000200044F80409202060700020A0702070DFE70120EFE72068806936EA000004D06B
:207AC0000020B842CFD00020D4E70120F9E770B516460D4604461EE0324629462046FFF7B2
:207AE000EBFE08B1012070BDFEF74AFC801BA84200D885B920688069C04380060BD554F89A
:207B0000440F40F0200044F80409202060700020A0702070E6E720688069C0438006DBD433
:207B2000002070BD70B516460D46044620E0324629462046FFF7C0FE08B1012070BD681C4E
:207B400016D0FEF71DFC801BA84200D885B920688069C04380070BD554F8440F40F02000CC
:207B600044F80409202060700020A0702070E4E720688069C0438007D9D4002070BD00002C
:207B80000F4810B50D4901601421416000214FF480328160C0E90312416101760122427693
:207BA0008176C27601774177FDF7A4FF002803D0BDE81040FDF71ABC10BD000000640040A4
:207BC0004C000020094808B5816C41F001018164806C002200F00100009011460F20FEF71C
:207BE000D7FDBDE808400F20FEF7C4BD00100240F0B587B014216846FBF751FD1D48C16C3C
:207C000041F08001C164C16C01F080010591C16C41F00201C164C16C01F002010591C16CEE
:207C200041F00101C164C06C012200F00100D4034FF09046059021463046FEF79BFB0E4F66
:207C4000012238213846FEF795FB009401240025694630460194CDE90245FEF79BFA38202E
:207C6000CDE9000469463846CDE90245FEF792FA07B0F0BD0010024000040048134810B57D
:207C8000114901601249416000210122C0E90212016141618161C1610162FEF7CBFB08B14D
:207CA000FDF7A4FB00210948FEF770FB08B1FDF79DFB00210548FEF794FB002803D0BDE888
:207CC0001040FDF793BB10BD0058004074000020E49CD1100D4810B50B4901604FF4E13194
:207CE0004160002181600C22C160C0E904128161C16101624162FFF7BBFC002803D0BDE87C
:207D00001040FDF773BB10BD00380140C8000020FEE7FEE7704700002DE9F041444C054620
:207D20008846E0680026810728680DD0E16801F00301814216D1A8B1E0686968C0F30210F3
:207D4000401C88420ED120E0012804D0022805D0032807D108E02168890701E02168490566
:207D6000002907DB01265FE02168890302D421684903F5E7E1686A686FF00F0321F07301E5
:207D800003EB021211430143E160206820F080602060FEF7F5FA074605E000BFFEF7F0FA5C
:207DA000C01B022837D820680001F7D4B8F1000F18D0B8F1010F1DD0287D4FF07E4140082A
:207DC00001EB4060A96840EA01202169194A114008432061206840F080602060FEF7D0FADA
:207DE00007461AE0A868297B000240EAC1602169114AECE7288A1149400801EB4050A968A2
:207E000040EA012021690E4AE1E700BFFEF7B8FAC01B022801D9032606E020680001F5D5C6
:207E20002069A969084320613046BDE8F081000000100240FF80FFF9FF80FF070000E0FF22
:207E4000FF809FFFF8B51C4D06460024A86DC00002D5FEF703FD0DE0A86D40F08050A865CF
:207E6000A86D00F080500090FEF7F8FCA96D21F08051A965B0F5007F04D0802E07D94FF0E9
:207E800003040AE0802E08D9A02E01D804E001D1022402E0702E00D101240848016821F09F
:207EA000070121430160006800F00700A04201D00120F8BD0020F8BD001002400020024084
:207EC0007047FEF707BC10B596B044216846FBF7E6FB142111A8FBF7E2FB4FF40070FEF7DD
:207EE00089FC08B172B6FEE70120032400900004019002201421CDE90A04CDE90C41072184
:207F0000CDE90E1010906846FEF722FF08B172B6FEE70F20CDE9110400201390149015905D
:207F2000042111A8FEF7FCFD002801D072B6FEE716B010BD0248016841F47001016070476B
:207F400088ED00E090F82410090706D501684A68436B22F400421A434A6090F82410C90771
:207F600006D001684A68836A22F400321A434A6090F82410890706D501684A68C36A22F44F
:207F800080321A434A6090F82410490706D501684A68036B22F480221A434A6090F824103D
:207FA000C90606D501688A68836B22F480521A438A6090F82410890606D501688A68C36BF0
:207FC00022F400521A438A6090F82410490611D501684A68036C22F480121A434A60016C5B
:207FE000B1F5801F06D101684A68436C22F4C0021A434A6090F82410090606D501684A68FB
:20800000806C22F4002202434A6070472DE9F84300260446C0F88460FEF7B2F9804620684B
:2080200000684FF0200500076FF07E4712D54346002229042046009700F036FB50B12168E2
:2080400051E8000F20F0800041E80002002AF6D1E56721E020680068400722D54346002206
:208060004FF480012046009700F01EFBC8B1216851E8000F20F4907041E80002002AF6D1BC
:208080002068083050E8001F21F0010140E80012002AF5D1C4F8805084F878600320BDE8E4
:2080A000F883E567C4F8805044F8606F666026760020F4E738B5054600206854052235A1F4
:2080C0002846FBF77FFA354C98B1082234A12846FBF778FA002827D0062234A12846FBF7B0
:2080E00071FA00283DD02946BDE8384031A000F05BBB6A4635A1681DFBF7A0F901282BD1C2
:20810000FDF730FA606000889DF80010884209D00A4601462EA000F047FB60689DF80010AD
:20812000018017E033A019E06A4628A105F10800FBF784F901280FD19DF80010617034A0C2
:2081400000F032FBFDF70EFA6060C27861788A4203D0C170FDF72EFA38BD34A000F024FB6F
:2081600038BD6A4619A1A81DFBF768F90128F7D19DF80010A17035A000F016FBFDF7F2F92C
:2081800060608278A1788A4201D08170E2E735A0E4E7000053455449440000003C00002040
:2081A0005345544445425547000000005345544449520000556E6B6E6F776E20636F6D6DE5
:2081C000616E643A2025730A000000002578000043757272656E742049443A2030782530EC
:2081E00032582C204E65772049443A203078253032580A0043414E20494420756E63686139
:208200006E6765643A203078253032580A000000536574206465627567206C6576656C3A10
:20822000203078253032580A000000004465627567206C6576656C20756E6368616E676505
:20824000643A203078253032580A000053657420646972656374696F6E3A20307825303239
:20826000580A0000446972656374696F6E20756E6368616E6765643A203078253032580A43
:208280000000000010B5806AFFF770F810BD70B5846AE06FD4F8805021688968090604D5A4
:2082A000212802D1204600F0A2F820688068400604D5222D02D1204600F073F8D4F88400F0
:2082C00040F01000C4F884002046FFF74FF870BD10B50146806A0A68126892062BD402686B
:2082E00052E8003F23F4807342E80034002CF6D10268083252E8003F23F0010342E8003418
:20830000002CF5D10268083252E8003F23F0400342E80034002CF5D12022C0F88020026E9E
:20832000012A08D1036853E8002F22F0100243E80024002CF6D100224266026E012A02D0C7
:20834000FFF74EFA10BD09684968B0F8582089B28A4201D9A0F85A10B0F85A10511A89B235
:20836000FEF7BAFF10BD10B50246806A01214166016E012902D0FFF734FA10BDB0F8581056
:208380004B08A0F85A301268526892B2914201D3A0F85A20B0F85A20891A89B2FEF79CFFA7
:2083A00010BD016851E8002F22F4907241E80023002BF6D10168083151E8002F22F00102AA
:2083C00041E80023002BF5D1016E012908D1026852E8001F21F0100142E80013002BF6D1DA
:2083E0002021C0F880100021016681667047026852E8001F21F0C00142E80013002BF6D10A
:208400002021C167704700002DE9F0410446016880682269E3691043626900251A43104390
:20842000714F0A68714B1A4002430A6020684168E26821F44051114341602168A069B942A2
:2084400001D0226A10438A6822F4306202438A606749236867488B420DD1D0F8880010F0BE
:20846000030006D0012847D0022843D0032830D144E001212EE060498B420BD1D0F8880084
:2084800010F00C0034D0042836D0082832D00C281FD133E059498B420BD1D0F8880010F096
:2084A000300025D0102827D0202823D0302810D124E0BB420DD1D0F8880010F4406017D03A
:2084C000B0F5806F18D0B0F5006F13D0B0F5406F14D010214A4A00264FF40040BB422FD186
:2084E00071B102290FD004290FD0082973D10FE00021EFE70221EDE70421EBE70821E9E702
:20850000FEF7B0FB03E0104602E0FEF7CFFBE8B3626802EB420181425DD8B0EB023F5AD846
:20852000010E03025008181871410023FAF7F4FE344AA0F5407191424DD82168C8604BE04F
:20854000E3694FF6EF77834228D1092943D2DFE801F005080B420D4242421000FEF782FBB8
:2085600006E0FEF791FB03E0104602E0FEF79EFB60B14100606801EB5001B1FBF0F0A0F177
:208580001001B94227D84FF6F07100E024E00140C0F3420001432068C1601DE009291AD208
:2085A000DFE801F005080B190D1919191000FEF759FB06E0FEF768FB03E0104602E0FEF7D3
:2085C00075FB48B1616800EB5100B0FBF1F0A0F11001B94205D90125A6662846E666BDE895
:2085E000F08180B2A9E7000000800040F369FFEF0038014000100240004400400048004067
:208600000024F400FFFC0F0070B54165A0F8582000210446C0F884102220C4F88000606F59
:20862000D0B11E4BC362636F1D481863636F1D485863606F13468163656D21682A4624315B
:20864000606FFDF77FFC38B11020C4F884002020C4F88000012070BD206940B1216851E87D
:20866000000F40F4807041E80002002AF6D12068083050E8001F41F0010140E80012002AFD
:20868000F5D12068083050E8001F41F0400140E80012002AF5D1002070BD0000D1820008B9
:2086A000678300088F8200082DE9F047994617460D4604464FF00008089E33E0701C31D0FC
:2086C000FDF75EFEA0EB0900B04218D8BEB120680168490726D5802D24D0402D22D0C169FF
:2086E000C94309070DD4082505622046FFF759FEC4F8845084F878800120BDE8F0870320D2
:20870000FBE7C069C04300050CD421684FF4006008622046FFF745FE2020C4F8840084F835
:208720007880ECE72068C06935EA000004D00020B842C3D00020E0E70120F9E710B5044824
:2087400000F00AFABDE810400148FEF72DBE0000C8000020FEE703B401984100009850EAD7
:20876000C12018BF04204A0D18BF40F0010040F2FF72B2EB515F08BF40F00200012808BFE5
:20878000052002B070470907090E002804DB00F1E02080F80014704700F00F0000F1E020F9
:2087A00080F8141D704700000FB4802110B503AB0648029AFAF728FE82B24FF47A730349D1
:2087C0000348FFF70FF810BC5DF814FB98010020C800002030380A2801D20120704700201B
:2087E00070470000B5EEC00AF1EE10FA02D89FED0E0A7047401AB0F5006F02DDA0F5805085
:2088000004E010F5006F01DA00F5805000EE900A9FED061AF8EEE00A20EE811AC1EE000AFA
:20882000B0EE600A704700000000000000008039034610B50020024604E09C5C521C20449C
:20884000C0B2D2B28A42F8D310BD000000B58BB000200121CDE90601039005900090019086
:2088600002900891049069460D48FCF73DFF08B1FCF7BCFD0A48FDF717FA08B1FCF7B6FDEB
:2088800002210748FCF7C0FE08B1FCF7AFFD0520FDF792FB03A0FFF787FF0BB000BD000020
:2088A0004C00002043414E3120696E697469616C697A6564207375636365737366756C6CC7
:2088C000790D0A00F0B587B00025CDE9000508200295CDE903500E468DF814500D4C4FF4AB
:2088E0007A7709E02068401C2060B84204DD4FF0FF30256007B0F0BD0748FCF7E7FF0028B8
:20890000F0D006AB3246694603482560FCF78EFE0020EFE7300000204C0000200748016806
:208920000A6842F010020A600068016841F020010160202202490148FEF72EBFC8000020F3
:20894000340200202DED028B82B04FF0FF3B9FED5C8AFDF7C7FEFFF7B6FAFFF749F9FFF770
:2089600031F9FFF70DF9FFF789F9FFF7B3F9FFF76DFFFFF7D3FFFCF7F5FD0546018851A0E3
:20898000FFF712FFA97856A0FFF70EFFE9785BA0FFF70AFFDFF88491A978DFF884A189F8D1
:2089A0000010E9788AF800105E4F07E05E4505D096B1012E51D0022EF8D176E0FCF7D2FC01
:2089C00038B108213846FDF7CDFC6420FDF7F4FAF4E7FCF7B7FC8046012208213846FDF7DF
:2089E000C9FCFDF7CDFC0646FCF7ACFC04460A20FDF7E2FAFDF7C4FC861B0FD000EE106A2E
:208A0000B8EE400ADFED480A4146204620EE200AFFF7E8FEDFED450A20EE208A99F80000E3
:208A2000A04620B1C8F10000B1EE488A84B29AF8000060B118EE100A00F0EEF841EC100B3E
:208A4000214653EC102B3AA00096FFF7ADFE10213846FDF787FC0126ABE79FED3E0A002150
:208A6000009128EE000AAA228DF800200191BDEEC00A220A8DF8012010EE100A8DF802401C
:208A80008DF80400020A8DF805108DF806108DF8032007216846FFF7CBFE8DF80700288893
:208AA0006946FFF70FFF28B1022620213846FDF759FC7BE7012220213846FDF75BFC8BE7F9
:208AC0000000000043757272656E742043414E2049443A203078253032580D0A000000001C
:208AE00043757272656E7420446972656374696F6E3A203078253032580D0A00437572723E
:208B0000656E74204465627567204C6576656C3A203078253032580D0A0000003E00002099
:208B20003D000020000400486F12833A0000B443416E676C653A2025752C2056656C3A20AF
:208B4000252E32662064743A202575206D730D0A000000000000C84210B50446016811484C
:208B600081421ED1C869C043C0061AD4102008622046FEF7B3FB0C4800684068C0F1200083
:208B8000C1B20A4801700A48FFF794FA20210848FAF763FD2046BDE8104020220449FEF708
:208BA000FBBD10BD00380140500100203C0000203402002010B500290AD00878002807D04D
:208BC00005487844FBF7B6FF002801D0002010BD0248784410BD0000AE020000A6020000D4
:208BE00010B500290AD00878002807D005487844FBF7A0FF002801D0002010BD02487844A8
:208C000010BD00009E020000960200000808A0F500114FEA3101704743004FEAD30C4FEAE3
:208C20003C0C43401FBF40070CF1605113F0FE4F70471CF0006F03D100200CF0004170472C
:208C40000CF0004343EA507010B540EACC0000F00EF800BF000000924FEA0001FFF7D6BF21
:208C60004FF000414FF00000A1F5002170470EF1020E2EF0030E5EF8044B244204D44FEA6D
:208C80004102B2F17F4F11D84FEA4003B3F17F4F0CD80ED14FEAD07CB2F17F4F0CEB4C0C41
:208CA0000CF1020C08BF4CEBD17C04E04FF0080C01E04FEAD17C0CEB4C0324FA03F404F071
:208CC0000704B4F1040C06D20EEB840CBDE810404CF0010C6047DFE80CF0070802024FF079
:208CE0000040A0F5800010BD0846420018BFD2F1807288BF00F0004010BD4FF04070E1EE34
:208D0000100A7047FBF772B9FBF7A6BA00000000000000000102030406070809A0860100C4
:208D2000400D0300801A060000350C0040420F0080841E0000093D0000127A000024F40065
:208D400000366E010048E801006CDC02000000000102030400000000000000003031323323
:208D60003435363738394142434445464030580030313233343536373839616263646566ED
:208D800040307800040000080000000000000002000100001030313233343536373839615E
:208DA00062636465667870003031323334353637383941424344454658500000024000004B
:208DC000000000A00000000005400000000000C8000000000C4000000000409C00000000BE
:208DE000194000000020BCBE0000000034400000BFC91B8E00000004B5400000504BCFD0A8
:208E00006607E2CF010000006C4100003E8251AADFEEA73401000000D9420000DCB5A0E2F4
:208E20003A301F97FFFFFFFFB4450000FD25A0C8E9A3C14FFFFFFFFFFF3F0000000000803D
:208E400000000000FF3F000000000080000000009C8F0008000000204C000000C8310008B4
:208E6000E88F00084C0000206C080000E43100081C00000043000000F8FFFFFF0C00000016
:208E80000E0000000F0000002E0000001001000043000000F8FFFFFF00404040404040407E
:208EA00040404141414141404040404040404040404040404040404040050202020202025C
:208EC0000202020202020202022020202020202020202002020202020202909090909090D2
:208EE0001010101010101010101010101010101010101010020202020202888888888888F6
:208F0000080808080808080808080808080808080808080802020202400000000000000069
:208F2000000000000000000000000000000000000000000000000000000000000000000031
:208F4000000000000000000000000000000000000000000000000000000000000000000011
:208F60000000000000000000000000000000000000000000000000000000000000000000F1
:208F80000000000000000000000000000000000000000000000000000000000001000000D0
:208FA0001000000000000000000000000000000000000000000000000100000000000000A0
:208FC000000000000000000000093D0000000000000000000000000000000000000000004B
:088FE000000000000000000089
:040000050800018D61
:00000001FF
